:020000041100E9
:10300000002373B52B4D2C4C28006361022601F080
:1030100065F94021FE2221742800284B009601F01A
:10302000AFF9002836D1217CFF222800244B0096DE
:1030300001F0A6F900282DD1224BA2899A4226D16F
:10304000E389214A93420DD1204B6361204B2268D2
:10305000002A03D1002B01D043CB43C4280001F048
:103060007BF973BD1B4A934201D00023EFE71A4B53
:103070001A4A1B68934206D9C02304222800217CE7
:103080009B0001F0F3F9114B6361154BDFE700235F
:103090002374EAE7CC233821AC2228009B01217459
:1030A00001F0E4F90028F2D10E4B63610E4BE3818D
:1030B0000E4BCCE7A442FF1F6462FF1F7062FF1F2C
:1030C0007262FF1F59590000830500000941001179
:1030D0002CB90011821500008862FF1F87130000C1
:1030E00038B90011C1410011AAAAFFFF20B900118F
:1030F000F7B5164B0192C318021D002000938823D8
:103100005B05D3181B685C1C1AD09CB2402C18D8E5
:103110008D781E0CAC466746CD782D023D43AE42FD
:1031200006D1019800280ED110000C70240A4C70B2
:1031300003249BB20733A343D218009B9A42DED3E9
:10314000FEBD4432F9E71000FAE7C046FC0F00006C
:10315000802213B503000324019189B25201073183
:103160009B18A14304305A1A88235B05C3181B68B7
:10317000591C03D190429241104016BD99B240298A
:1031800007D80B000733A343C0189042ECD30020AC
:10319000F3E74430F9E7134B134A1B68126810B584
:1031A000FA24934201D81A00F824104BE4021B6859
:1031B0009A4210D813000E4A12689A420ED3013375
:1031C00007D1F823DB029C4203D10A49054808F0E5
:1031D00083FA200010BDFC24E402ECE7FE24E402A4
:1031E000F7E7C04600C0071100D0071100E0071143
:1031F00000F00711FFFFFF7FF0B59BB015000490B2
:103200000391402A00D9A0E006AB59801A80FFF74D
:10321000C2FF0400042816D9002206A9FFF768FFA0
:10322000052810D906AB1B88AB420CD1002D07D066
:10323000514B2A000499C01808F0E6F9002802D181
:1032400001201BB0F0BD06AB1D8020000699FFF7E2
:103250007FFF041E7BD1069B0793FFF79CFF802313
:103260005B01C618802307001B039E4201D3F8268A
:10327000F60288235B05F31801931B68013302D023
:10328000019808F0D9FA3D49019808F025FA3B1D4C
:103290000293331D05938822029B52059B181B68DD
:1032A00008935A1C3CD044219AB20091402A04D879
:1032B0000320D11D814389B2009103991B0C8B42DD
:1032C00024D0402A22D80122300008A9FFF710FF9D
:1032D000021E1BD1380008A9FFF70AFF04000428CA
:1032E00031D9009A059B9B1880225201B218934253
:1032F00040D288235B05C118009A09A808F00CF891
:103300001D4B009A09A9F01808F05EF9009A029B7B
:103310009446634402931A4B029AFB189A42BAD31A
:1033200088235B05FC1821680198013908F0D4F95D
:10333000200008F081FA039A07AB5A803000079901
:10334000FFF706FF0400002C03D1002079E70428D2
:10335000FBD988235B05E018069908F0BDF9032323
:10336000EA1C9A4300D16BE7034B0499E01808F07C
:103370002BF965E70424ECE704000011FFFFFF7F51
:10338000F80F0000F7B505001400402A21D80027E7
:1033900001AE71803780FFF7FEFE042816D93A008F
:1033A0003100FFF7A5FE042810D93688BC420BD0A7
:1033B000BD4209D0221CB44200D9321C064B92B245
:1033C000C118280007F0A8FF30B2FEBDC04300B20C
:1033D000FBE703204042F8E70400001137B5042260
:1033E00004000D0001A81649FFF7CCFF02000428D5
:1033F0000BD1019BA34208D3AB4204D0104901A8D2
:103400000195FFF7F9FE01203EBD0E4C2368200018
:10341000019308F011FA019920000139019108F097
:103420005BF980235B01E418074B9C42EED1042238
:10343000034901A80195FFF7DFFE0020E4E7C0463D
:103440005555000000C007110000081130B589B0C3
:1034500007F0EAFF10226946254808F03DF8254BA1
:10346000009A9A420ED1019B029A0F2B33D8002169
:1034700001240698013B08D2002900D00292029B49
:10348000013331D10023029325E0551CF2D1020013
:103490002100EFE710341022200004A908F01CF8E6
:1034A000029B013301D1069B0293882304995B059B
:1034B000C918059B06981A03120B049105928142C4
:1034C00003D02B4201D107F027FF019B013B019361
:1034D000019B002BDED1029B002B03D004930498A8
:1034E0004168084709B030BDE025014C2D03EFE7E6
:1034F00000000111504859368022F8B5964C974B80
:10350000D200002120001C6008F02EF82300944A0D
:1035100088331A60934B1A786A23002A00D011333B
:10352000E3620A232365904B37221B780820A363AC
:103530008E4B2118E361102323628D4B3B25636181
:10354000C823DB00A36123008C331A602823013ACF
:10355000E26320646364CA67043A211DCA672100DC
:10356000BC310D602100C03108602100C4310B6006
:1035700021000635CC310D602100083DC8310D60B9
:103580002100D0310A602200D43210602200D832EB
:10359000136022000227E032210017604222DC3152
:1035A0000A6021001B3DE4310D602100E831086014
:1035B0002100EC310B6023000521F4331960230056
:1035C000F0331A602300183290331A6023009433CA
:1035D000186023001E3A98331A60AF23DB00236083
:1035E000644BFA262363644B644DE360644BF03113
:1035F000A3642300FF31FC33B600A16021611E608B
:10360000A5627325E5656D3D6565A56596255D4AF1
:10361000AD00E264666258606766A566002709250A
:10362000A767E566584F594D606720002567E26738
:103630003A6015279C30676007001A203860200028
:10364000A0300700212038602000A83007004C4837
:1036500038602000F830066026006427A436376002
:1036600026005F3FAC3637602600033FB036376038
:103670002600C637B436376026000027B8363760D4
:1036800038269E60424E96205E64424E5A66DE6147
:10369000414E9A645E62F53EFF3E9E621E269A6728
:1036A000354A8000DE661F675F67DD651D6618624C
:1036B000DA67BE23394A5B00E250394BD8382350D1
:1036C00004302250C4225200A350C623E4205B00E1
:1036D000E1500433334AE1503349344BD16034492B
:1036E000800019503349E938FF3819503249043005
:1036F000195032493248D16132491163324951631C
:103700001900F4310860CE20304940001160304982
:10371000195019002F48F83108602F49D1658221CE
:103720002E4A89005A501A002D490832D1671A00D2
:103730002C49B432116088212B4A89005A501A0052
:103740002A49883211602A4ADA6407F06DFF0120A5
:1037500007F0CAFEF8BDC0460004FF1F0065FF1F4A
:10376000E06FFF1FD444FF1F4A0AFF1F3A07000003
:1037700080C3C9019A020000DC0500006A1800003D
:1037800050C3000088130000F009FF1F204E000006
:103790006509FF1F68100000C409000040420F00C7
:1037A00010270000FC00FF1F751CFF1F0000FF1FFB
:1037B000C92CFF1F5930FF1FF12EFF1F3520FF1F9F
:1037C0002527FF1F5120FF1FFD21FF1FC11FFF1FC6
:1037D0004929FF1F312AFF1F8D19FF1F5528FF1F81
:1037E0007925FF1F8525FF1FC11EFF1F791FFF1FA2
:1037F000391EFF1F0223F0B50124614D614E2B706D
:10380000614B91B01C70614F039333680021042019
:10381000BB7006F0F3FB042006F0EAFA002398429E
:1038200005D0BA78552A02D0332A00D09BE0336005
:10383000042006F05DFD07F067FFFFF75DFE07F06F
:10384000A3FE1F2201240021514B10AE1A70514BD0
:103850001C70514B1970514B19689143163A0A4329
:103860001A60602219689143403A0A431A6007F0CF
:1038700013FF07F051FEC120FF21494B80001A5869
:103880008A431A50C522920098588843BF39014391
:1038900099509858434908408021C901014380202C
:1038A00099509958C0050902090A0143995080218D
:1038B0003D48490107F0F8FE032322003B490194EB
:1038C00000933B4807F018FE2C223A4905A807F060
:1038D00023FD05AC61782078023406F0A9FAA642EF
:1038E000F8D1354C1120002106F0B6FB2268334B8D
:1038F00003201A40A023DB021343236080232268A5
:103900009B041343236022682D4B1A4080239B03A2
:10391000134323602B4A2C4B934200D8012007F01D
:103920007BFF07F019FD80232268DB04134323602B
:10393000287807F029FF039B1878C0B207F054FFDE
:1039400007F022FD2149042007F096FD06F09CFCBB
:1039500000F03EF800F0B6FD00F05EFE00F002FA66
:10396000002011B0F0BD00932100184A042007F098
:10397000EBFD8023DB059C62FFF768FD58E7C0463E
:103980004A0AFF1F34F00040D444FF1F9462FF1F17
:10399000480AFF1F490AFF1F680AFF1FBCF00040CA
:1039A00000E100E0FF00FFFFD844FF1F5C57FF1F4E
:1039B000D854FF1F48B8001114F00040FF7FF8FFF3
:1039C000FFFF9FFF0080FF1FE06FFF1F3B0001080C
:1039D000002210B51100112007F026FC10BD0000D8
:1039E000002370B50925334E334C3362E368112050
:1039F000AB43E36007F088FD112007F0FDFC1120C8
:103A000007F09AFC4023226811201343236080238F
:103A10006268DB02134363608023A2681343A360E0
:103A2000A368264A1340A3608023A2689B01134326
:103A30001022A360236C934323640123226C1A4356
:103A40002264802252003262216B1D4A11402163A0
:103A5000616B11406163A16B1140A163E16B0A408E
:103A6000E263E26817490A40E260174A11680B43B3
:103A7000136007F0E9FBFD21144B154A89005A50E9
:103A80008023C720626B5B0313436363E36880009A
:103A90001D43104BE56019580F4A11408022120255
:103AA0000A431A50802292051A6008220B4B5A636F
:103AB00070BDC04600F000403CF00040FFFFDFFF5B
:103AC000EFFFEFFFFFFF7FFF003800400000FF1F08
:103AD0005118FF1F00E100E0FF00FFFF000005405C
:103AE00070B5284C238C002B23D0228A002A21D1A8
:103AF000DA0023826382A382E38223836383A38326
:103B0000E38322606260A260E2601F4D1F4A64206E
:103B1000EB8093420AD8FA220020D200934205D9C2
:103B20001B4A0A21981807F07FFEC0B200232872B2
:103B3000238470BD0720E11CCA7F01320240CA778E
:103B400005D10325201DC17F01312940C1770832ED
:103B50005200A352002321001A00088A01321B18C8
:103B60000231082AF9D1221DD27F9200A350626847
:103B700023689B18A2689B18E2689B185B099BB29C
:103B8000C3E7C046D461FF1F7C62FF1FB70B000074
:103B900030F8FFFF30B503A804880B20002C0ED1AD
:103BA0004968074D08784978090201430A20A9426B
:103BB00005D1012120001980024B1B7A137030BD02
:103BC000192A00007C62FF1FF7B5150008AA1688A5
:103BD0004A680F4F14785278120222430A24BA42DC
:103BE00014D10122DBB2019200962A0007F09CFA60
:103BF000041E0BD1074B1B68002B07D068782A786E
:103C00000002104342425041013098472000FEBD5F
:103C1000022900000062FF1F30B50125037904006E
:103C2000BFB02B4211D00A49408806F0E9FD284276
:103C30000BD0084B01A95B8D4D800B80064B0022F9
:103C40001B7A60880B7103F0BBFE3FB030BDC046ED
:103C5000F861FF1F1841FF1F7C62FF1F10B5054967
:103C6000054806F083FD0421044A054806F040FD9E
:103C700010BDC046F861FF1FFFFF000074B80011BF
:103C80001841FF1F10B5024804F01CFD10BDC046CE
:103C9000193C0011012303700B4B1A7A4270022267
:103CA00082709A78C270DA780271032242711A79AE
:103CB00082715A79C2710C2202729A794272DB794E
:103CC00083720B207047C0467C62FF1F022310B531
:103CD0000370013B43700533837010330371443B21
:103CE00043712A3383714433C37100230372064B3B
:103CF00004001B8843720A30FFF7CCFF831D0A3093
:103D0000C0B2E37010BDC0467C62FF1F10B5142026
:103D100007F0C2FB124B14220021186007F024FCAC
:103D2000002007F041FD012007F0CEFB022007F044
:103D300013FD032003F06AFF042005F07FFF052038
:103D400003F0A8F9062003F075FE072001F00CFA35
:103D5000082006F0ADFC092000F0E8FF10BDC046C9
:103D60000462FF1F07F080FA012007F0ADFC07F0A6
:103D700013FB0000094B10B50400984205D001293F
:103D800004D12000064906F0F1FC10BD0229FCD147
:103D9000013904F055FC0028F3D0F6E7FEFF0000DF
:103DA0002A62FF1F70B50D7A100004AA2C00168835
:103DB00010221440154220D1002E20D10A78022A68
:103DC00018D14A68517815780E4A09022943914260
:103DD00005D00D4A914209D01C800A2404E0142227
:103DE0000A491A8007F098FA200070BD0C22084991
:103DF0001A80F7E71C800124F6E70824F4E70B2477
:103E0000F2E7C046F3FF0000F4FF00006043FF1F2D
:103E100050B9001110B504000749084806F0A6FC87
:103E2000074804F08FFB0020E40704D50721054A6A
:103E3000054806F05DFC10BD2A62FF1FFFFF000071
:103E4000753D0011B8B800115C41FF1F00B50C4B67
:103E5000BFB01A780B4902A800F098FC6B4680B2FC
:103E6000D880002809D06A46074B01A91B88938097
:103E7000064B0022188803F0A3FD3FB000BDC046EA
:103E80000862FF1F0962FF1FB641FF1FC042FF1FEC
:103E900000B50C4BBFB01A780B4902A801F0D6FC54
:103EA0006B4680B2D880002809D06A46074B01A92A
:103EB0005B8D9380064B0022188803F081FD3FB094
:103EC00000BDC0463262FF1F3362FF1F5C41FF1F0F
:103ED000C042FF1FF7B50E00377A1C0008AB110077
:103EE0003D001A8820231D401F423CD13378022B0D
:103EF0003BD173681F785B781B023B431E4FBB426C
:103F000008D01E4FBB4214D01D4DAB4221D00A2514
:103F10002800FEBD002A2AD1142C2AD82200F068DD
:103F200007F0FAF9174B1C70012CF1D9FFF7B0FF1D
:103F3000EEE7002A1BD1202C1BD82200F06807F0E6
:103F4000EBF9114B04211C70104B187807F064FA40
:103F5000DEE7E3B20124009201940A00310007F089
:103F6000E3F80500D4E70825D2E70125D0E70B25C3
:103F7000CEE70D25CCE7C046F3FF0000F4FF0000BC
:103F8000022900003262FF1F0862FF1FB462FF1F98
:103F9000332310B5040003700A220749013007F0EB
:103FA000BBF9064B0F201B681A0AE37222731A0C26
:103FB0001B0E6273A37310BD7C62FF1FA462FF1F00
:103FC00030B5012503790400BFB02B4213D00B4953
:103FD000408806F015FC28420DD06A46084B02A81E
:103FE0001B889380FFF7D4FF6B46D880002260883F
:103FF00001A903F0E5FC3FB030BDC0462A62FF1FB7
:10400000B641FF1F10B5024804F05CFB10BDC0466E
:10401000C13F001170B5160004AA148805AA1578CE
:104020004A685078117800022A4A08438018052807
:104030004BD807F019FA03131E29343F0720032C2D
:104040000BD80422121BAA4200D92A0022491A8046
:104050003000091907F060F9002070BD0720112C0D
:10406000FBD81222121BAA4200D92A001B491A802F
:10407000EEE707200E2CF0D80F22121BAA4200D91F
:104080002A0017491A80E3E70720032CE5D8042209
:10409000121BAA4200D92A0012491A80D8E7072029
:1040A000032CDAD80422121BAA4200D92A000E4996
:1040B0001A80CDE70720032CCFD80422121BAA4276
:1040C00000D92A0009491A80C2E700220A201A8072
:1040D000C3E7C046DCD5FFFF03B900115062FF1FE4
:1040E000F3B80011EEB80011E9B80011E4B80011FE
:1040F00010B50D21024A034806F0FAFA10BDC04679
:10410000D8B80011CC41FF1FF0B50024274E85B070
:104110003000B47100F0E2F8254D264BEA89297C85
:104120009A422FD10423300003AA00F057F904006B
:10413000300000F011F90123B371002C34D16B462B
:1041400099892B68C9BA4B4329891B4A1B145B18F0
:1041500053806B46D9896B6849BA89B24B436989E8
:104160001B0C5B181548191C1BB2834200DD011C97
:104170000B0400D5002113889180013313802000A7
:1041800005B0F0BD0227220003AB3000009700F01D
:10419000F7F80E230400297C0122300000976B44BD
:1041A00000F0EEF80443C3E71C00E8E7A442FF1F59
:1041B0006462FF1F830500007C62FF1F0F27000061
:1041C00073B5234E300000F089F8224D07236A466C
:1041D0003000297C00F002F904003000002C33D1BB
:1041E0006B461B787F2B2FD800F0B6F86B46D8783B
:1041F000F02302041B031A406B469B8816495BBAE6
:104200009BB21A432B68000953432A891B0C9B1845
:104210004B806B465A789B7812031B011A436B68DC
:10422000024353436A891B0C9B180C481A1C1BB28F
:10423000834200DD021C130400D500220B888A8013
:1042400001330B80200076BD00F086F80124F9E7E9
:10425000A442FF1F6462FF1F7C62FF1F0F27000044
:1042600070B5114C237C002B0FD0382B0ED10F4D85
:10427000280000F033F8CC23AC222800217C9B01DD
:1042800000F0F4F8280000F067F870BD084BE289F0
:104290009A42FAD1054D280000F020F800222800AB
:1042A000217C00F0C5F8EDE76462FF1FA442FF1F08
:1042B0008305000010B5084B1A7C002A09D05B6901
:1042C000002B06D09847041E01D0FEF799FE20006F
:1042D00010BD0124F9E7C0466462FF1F70B5C179C3
:1042E00005000C00631E9C411A4BE402E4184900CF
:1042F0000460C9B2007905F0E5FEE9796879490002
:104300000131C9B205F0DEFEE8790930C0B207F02C
:1043100013F80023E36661332360AA795B3B002A2C
:104320000ED022689A43023B134323600A23E361C1
:104330000733236200232363A3630133E36370BD68
:1043400022689A43022313432360462363610633A2
:10435000A361EFE70050004070B50025040003683A
:10436000DD66C0790930C0B207F0CEF829002079A7
:1043700005F044FE2900607905F040FE70BD0000A4
:10438000F8B51E0006AB1D78002304681700E3662D
:10439000616007F049F801238022E3662B00276162
:1043A0005200013B08D207F017F808200A4A1168AA
:1043B000002D03D12800F8BD2261F2E7236F0342EC
:1043C00003D02369013D3370013613685B1A032B58
:1043D000EED90125EEE7C0466008FF1F70B51C004E
:1043E000002305681600EB66696007F01DF80123DD
:1043F0008022EB6623005200013B08D206F0ECFF5E
:1044000008200A4A1168002C03D1200070BD2A61DF
:10441000F2E72B6F034203D02B69013C3370013666
:1044200013685B1A032BEED90124EEE76008FF1F27
:10443000002370B504681500E366616006F0F4FFC0
:104440000123E366256106F0C7FF8020064A80004D
:104450001168636B034205D113685B1A032BF8D90B
:10446000012070BD0020FCE76008FF1F70B51D0033
:10447000002304681600E366616006F0D5FF01239F
:10448000E36626610F33626B1A42FCD02B0A23616C
:104490001023626B1A42FCD0EDB2256106F09CFF3E
:1044A0008020074A80001168636B034205D11368BE
:1044B0005B1A032BF8D9012070BD0020FCE7C04631
:1044C0006008FF1F10B5084CE368002B08D180225C
:1044D000064B52021B689B186360054B1B682360E8
:1044E00006F0E2FEA06010BDA462FF1FC8F000400D
:1044F000CCF0004070B5184A936A916A9942FBD19A
:1045000016498A689A421FD39A1A8B60144B012667
:10451000186893B2D202D20E4343424300204C6843
:104520001B0A1B1912029B180E4C0A684B60551C83
:10453000A3420CD8002801D04B600A600A4A1360DD
:1045400008680A4B186070BD581E821ADDE7084AD9
:1045500030009B182A00EAE700F00040A462FF1F29
:10456000140AFF1F40420F00C8F00040CCF000408A
:10457000C0BDF0FF70B51F4C23793F2B01D93F23FD
:1045800023711D4B22791A701878C0B206F044FED0
:1045900018231A491A4A0B801A4913800B8053803A
:1045A000A379194980200B800C21938001334B4360
:1045B000164D191C0001834200D9011C2980D180AD
:1045C0006379002B11D101336371237A012B01D858
:1045D000022323726279237A0D4853430A215843F8
:1045E00007F022F90B4D286070BDA02BEDD9A02358
:1045F000EAE7C0469862FF1F480AFF1FBE42FF1F3E
:104600008044FF1FBC42FF1FBA42FF1FB842FF1F7A
:10461000710200008862FF1FF8B514210020FEF728
:10462000DDFE114C011E114D09D10C22104BC1CBE6
:10463000C1C4280006F098FFFFF79CFFF8BD0C22CC
:1046400020000C49FEF79EFE0C2802D0084B43CBFD
:1046500043C40C2228000849FEF794FE0C28EBD036
:104660000C220021E5E7C0469862FF1F6462FF1F2D
:1046700044B90011FC0C0000F50C0000F0B51D4C15
:104680008022A5440400882069465201400506F0B6
:10469000ABFE902212016A441300200032C832C3DC
:1046A00016C816C38023144C144FA6689B033343CB
:1046B000A3603B6007F020F88823A0685B05C01862
:1046C00007F0BAF80025882329008022A0685B053E
:1046D000C01840196944520006F076FF8023013566
:1046E000FF355B019D42EED1A6603E60044B9D44C8
:1046F000F0BDC046FCEFFFFFF043FF1F9808FF1F0F
:1047000004100000F0B5040087B0002825D06846EA
:1047100006F052FE1B4C022806D1062269462000F4
:1047200006F072FF002816D06946002301250F26E7
:104730002F00E25C013310091030874038002F0051
:10474000324097403A0002434A610439062BEFD1C8
:104750006846FFF793FF07B0F0BD182269460A4884
:1047600006F042FE6A46A300D358013305D0182252
:10477000FF21684606F0F8FEEAE70134062CF1D185
:10478000E9E7C0466509FF1F00090011F0B50025E3
:1047900004000E0085B0AA4200D183E04B1C0878CB
:1047A00001934B788978377909021943F3783F06EA
:1047B0001B040B431F43039720706570252800D10D
:1047C00093E033D8112813D806F076FE66000D0169
:1047D0000D010D010D01A700B500AE000D010D0189
:1047E0000D010D010D010D010D010D01E700070186
:1047F000232800D1C0E0DB2800D016E1042A00D82D
:10480000A9E01025052A05D0551F2A003800711D82
:1048100006F082FD05223100200006F07DFD2A0011
:104820003900601D06F078FD05353BE0562856D06E
:1048300010D8332800D19AE0552836D02628DAD16E
:10484000894B2900132218001D0006F08DFEFEF78B
:10485000D7FB59E0712800D174E0722800D17DE0C7
:10486000DC28C8D1022A00D875E07378BFB2637023
:10487000B378A370032A05D0033A390092B2F01C32
:10488000FEF7BAFC10223900E01CFEF77BFDC51CC8
:10489000002807DA60705CE00C222000734906F003
:1048A0003BFD0C25280005B0F0BD013A704D0C2AE7
:1048B00013D8002A0AD02800019906F02DFDFFF731
:1048C00059FE0C2228006B49FEF796FC29000C22A9
:1048D000601C06F021FD0D25E4E70C22EBE7644D9A
:1048E000654B2A0043CB43C2E9E7013A5E4D0C2AEF
:1048F00011D8002A08D00199280006F00DFD0C22DD
:1049000028005E49FEF778FC29001322601C06F09F
:1049100003FD1425C6E70C22EDE705225849601C6B
:1049200006F0FAFC0625BDE712225649601C06F087
:10493000F3FC1325B6E708225349601C06F0ECFC93
:104940000925AFE77178F02905D8504B188801F098
:10495000D9FB0225A6E7FF236370FAE74C4B012A37
:1049600003D072785A706270F3E75B78F4E7200046
:10497000FFF70EFB050095E7042A04D9454D2F608B
:1049800006F092FCA860FFF7B5FD0422039003A98E
:10499000601C06F0C1FC052584E73F4D062A15D9A9
:1049A00006222800019906F02FFE00280ED00622CC
:1049B0000199280006F0B0FC062238492800FEF7CD
:1049C0001BFC0123324A51780B4353702900062205
:1049D000601C06F0A1FC072564E7012ABBD07078B3
:1049E000FFF790FEB5E7012800D004E7931E2C4F97
:1049F000132B04D87378002B09D100F009F9294B47
:104A000039001D78601C6A1E06F086FC4AE7551EB8
:104A10002A000199380006F07FFC2349AAB2380029
:104A2000FEF7EAFB00F02CF9E9E7DA2893D1042A33
:104A300091D9082A15D9B37972791B021343F279F7
:104A400012041A43337A1B0613433B603B6805226A
:104A500031002000039306F05FFC0422601D03A9CF
:104A60006CE7FE236370F1E76462FF1F50B9001129
:104A70009862FF1FFC0C000044B90011F50C000007
:104A80007062FF1F5062FF1FF443FF1FC042FF1FF1
:104A90009462FF1FA462FF1F6509FF1FADAC0000F9
:104AA0009564FF1F9364FF1FAEDE00007047000097
:104AB000020010B5094B0A32094C92B2DA815A82CF
:104AC00098811882207802F083F90422054B012195
:104AD00020781A7006F0A0FC10BDC0467E43FF1F70
:104AE000DE64FF1FDD64FF1F013870B5042809D89C
:104AF00006F0BAFC0309230812001E4B02211878A5
:104B000006F08AFC70BD1B4B0821187806F00CFCDF
:104B10000022194B1A72F5E780220024164B154D1E
:104B200052001A81082128781A68DC7206F06CFCA1
:104B30002100287806F088FCE4E70E4B082118785D
:104B400006F0F2FB0D48FFF7C1F80D4B0D4A9B79BB
:104B500093800D4A13800022074BDA720132FF3234
:104B60001A810A4B5B78002BCCD0094A136006F0FF
:104B700043FEC7E7B462FF1F8862FF1FC942FF1FE1
:104B80009862FF1F8044FF1FBA42FF1F9462FF1FFD
:104B900034F0004010B5002904D1042802D10D30B2
:104BA00005F05AFA10BD000010B501290ED10428F5
:104BB0000CD10D3005F050FA054B1B78002B05D0B9
:104BC0002622044B04485A72FFF772FF10BDC046FC
:104BD000B664FF1F8862FF1FC40900000300F0B520
:104BE0000A4D8E18B14202D152008018F0BD0C78E7
:104BF0002F6824093C5D0F271C700C7801313C4064
:104C00002F683C5D5C700233ECE7C046B442FF1F86
:104C10000D22124B10B51A700C23114C1149237040
:104C2000093A033B1048637006F076FB2D230122FE
:104C30000E490F48A371FFF7D1FF01220D49FFF77D
:104C4000CDFF01220C49FFF7C9FF030000200B49EB
:104C500002001870FEF7D0FA10BDC046B264FF1F04
:104C60009364FF1F03B900119564FF1F6709FF1FBD
:104C70009A64FF1F6609FF1F6509FF1FAEDE000073
:104C800070B5124C142220001149FEF77BFB431E25
:104C9000104D132B17D8AB78002B14D0431C2B705E
:104CA00009236B7000230019037028782900013054
:104CB000C0B206F0F9FB297822000139C9B2002000
:104CC00005F034FC70BDFFF7A3FFEEE79564FF1F0E
:104CD000AEDE00009364FF1F10B5114B1A781870F8
:104CE000002A0ED000280BD10E4B1A78062A07D8BE
:104CF0005423D340DB0703D50B4B187802F068F838
:104D000010BD0028FCD0074B1B78012B02D0033BC1
:104D1000022BF5D8044B0121187806F07DFBEFE754
:104D2000B664FF1FDD64FF1FDE64FF1F70B54D4ECC
:104D30004D4A4E493070042005F084FA00211120BC
:104D400005F08AF9112005F06BFAFEF759F906F023
:104D500023FC032246494748FFF740FF2D24030068
:104D600004221C7044490130FFF738FF30230470DF
:104D7000424D434C437083702E3B06222000414934
:104D8000EB87FEF7FFFA062813D0200006F014FB8D
:104D9000022809D00321200006F04EFC8D23E37089
:104DA0006E3B237119336371062220003549FEF7EB
:104DB00023FA354B1B68FC335C64FFF761FF00206E
:104DC000FFF78AFF314C324A0121324B12782078AA
:104DD00001F0C0FF304A314B12780021207801F0F9
:104DE000B9FF01222E4B1A702E4B9B78552B31D1D7
:104DF0002D4B3B325A722D4B2D4AAB81EA812B82CF
:104E00006A822021307806F07FFA0120404205F0C6
:104E1000D9FB0120404205F075FCFFF769F9FEF768
:104E20001DFF00F0ABFC01204042FEF7F3FF012024
:104E300006F0E2FBF02001F049F90121307806F09C
:104E4000EBFA307802F020F91A4806F095FAFEF7EE
:104E5000C7FD70BD6422184B5B7953431A000A32B8
:104E6000CBE7C046B462FF1F954B0011A94B001160
:104E7000F443FF1F5062FF1F7062FF1F7E43FF1F3E
:104E80006509FF1FADAC00000065FF1FDE64FF1F5A
:104E9000E842FF1FC942FF1FB264FF1F9364FF1F58
:104EA0008464FF1F9462FF1F8862FF1FC409000013
:104EB000CE090000B662FF1F9862FF1FF8B50A0016
:104EC00020230D001A4019425DD05A4B1B78002B4D
:104ED00042D0FFF70FFB584B584C594E9968626807
:104EE000737A8A1ADB039A4202D36160FEF778FD77
:104EF000327A217A531EDBB2994230D1FFF7B0F9F2
:104F0000637A002B25D0013BDBB26372002B20D1EA
:104F10004C4B9B78552B01D106F06EFCE37A002BAD
:104F200012D00023A27AE3729A4202D0A372FEF753
:104F3000D7FD454A454F1388380001331380FEF7EB
:104F4000C5FE390006F078F9642370795843FFF7FD
:104F5000AFFD237A0133237220206840F8BD9142CF
:104F6000CED300272772FFF7A5F9A37ABB4202D060
:104F7000A772FEF7B5FD354F3800FEF7A7FE3900E2
:104F800006F05AF9BCE70BB2002B0ADA304B18785E
:104F900006F022FC002801D006F0CEFA80200002A4
:104FA000DBE70224214206D0244B01201A72FFF7CE
:104FB00093FE2000D1E70B071BD5FFF79BFA1E4B92
:104FC0001E491F4C98684A68637A821ADB039A422A
:104FD00002D34860FEF704FDFFF76CF9FFF740F9D4
:104FE00000F0E6FB2368DB0701D5FFF70BF808208C
:104FF000B3E7CB0609D5FEF773FD0E4B1B78002BEC
:1050000001D1FEF73FFE1020A7E70124214209D07D
:10501000104800F06DF806F01FFB2100112005F08C
:105020001BF8C6E7042408002040214296D0FEF772
:105030000DFFBEE7B664FF1FA462FF1F8862FF1F5B
:105040009862FF1F9462FF1F7C62FF1FC942FF1F0F
:10505000B462FF1FAC42FF1FF0B51B4B1B4F1B88F8
:105060003A8804001A4E1B4D85B09A420DD83288FA
:105070009A420AD3184B1A882B889A4205D1174AAC
:10508000174B12881B889A421BD0052001F074F838
:105090003B8802AA13803388019053802B88114DDE
:1050A00093800F4B02A91B88D3800F4B2A78188856
:1050B00002F090FD0D4B08212878019A1C7006F033
:1050C00073FA05B0F0BDC0468264FF1FBE42FF1FE9
:1050D000BC42FF1FBA42FF1F8064FF1F7E64FF1F98
:1050E000B842FF1FDE64FF1FC042FF1F7C64FF1F2A
:1050F00013B50C4B1C78002C11D1002801D00A4BA1
:1051000018600A4A0A4B11780A4A10780A4A019232
:105110000A4A0092002205F001F9200016BD112470
:10512000FBE7C046DD64FF1F7864FF1FDC64FF1FE0
:10513000CC64FF1FDE64FF1FB864FF1FBC64FF1F49
:1051400010B5064B12201B78052B06D1044B1322F9
:105150001988044B187801F0EBF910BDDD64FF1FCE
:10516000C042FF1FDE64FF1F10B500240122114B57
:1051700052421870104B1C70104B1A8001F084FFC3
:1051800004220F4B21001A700E480C3206F044FA2C
:10519000102221000C4806F03FFA07220B4B1C603E
:1051A0000B4B1C700B4B1C700B4B1A700B4B1C7079
:1051B00010BDC046DE64FF1FDD64FF1FC042FF1F3D
:1051C000DC64FF1FCC64FF1FBC64FF1FB864FF1FBB
:1051D0009264FF1F9164FF1FC242FF1F9064FF1F74
:1051E000F8B5174C0600257806A814240078052D7C
:1051F00023D1B41F134FA5B21824BD421DD88D1F53
:10520000ADB2BD4219D8FA256D00AA4215D21D00D3
:105210000D4F0A3DADB2BD420FD80C4C26800C4C50
:1052200021800C4900240A800B4A1380FFF714FFE9
:105230000A4B0421187806F077F82000F8BDC04624
:10524000DD64FF1F790C0000750C0000BE42FF1FDB
:10525000BC42FF1FBA42FF1FB842FF1FDE64FF1FA0
:10526000F0B50BB20D0089B0002B00DB70E1A44E4D
:10527000307806F0B1FA041E50D00378A22B00D18A
:1052800022E1D02B1AD0912B45D143780E2B42D15D
:105290009C4B82889A423ED19B4A83681278052AA9
:1052A00039D1032018567F2835D0984B1B68002B26
:1052B00031D05B68002B2ED098472CE080780728EF
:1052C00029D806F0D1F80428183F3F74A8D863788D
:1052D000002B0CD101218C4B19708D4B1A78002AB0
:1052E0005BD08C4B307801F035FD002855D007227B
:1052F000854B1A7051E061780029F8D1E378002BD2
:1053000011D0854A854B1278307801F023FD60700A
:105310006378002BEBD1200006F00EF9802000020C
:10532000684009B0F0BD784B1B78022BF3D0012107
:10533000307806F031FA0028EAD10121307806F001
:105340006BF8E5E76378002BD1D16F4F032807D1C5
:105350003B78052B02D101333B701EE00223FBE7B3
:105360006F4B1A886F4B0293002A0BD01B78002BCF
:1053700003D00121307806F017F93B78062B04D1D1
:10538000013BE9E7029B1A70F7E7042B41D10121A9
:10539000029B3078197006F03FF85C4B1B68002BBD
:1053A000B9D01B68002BB6D0574A107884E76378D1
:1053B000554F002B27D10622211D5B4805F0ACFF7D
:1053C00062895A4B5A491A80A2895A4B1A80E3893A
:1053D0000B800521397058490A80584A1380228A67
:1053E000574B1A80574B1B78012B09D11F2000F017
:1053F000C3FEFA22920042430421307806F0D4F82A
:105400000022484B75E7312B00D070E70022454B56
:105410001A700323A0E706220021434806F0FCF897
:105420000023454A04211380444A30781380444ABB
:10543000138005F079FF0821307805F075FFA37916
:10544000083B5A425341304A03331370304B1B78A8
:10545000002B06D0334B30781A78002A06D001F0A2
:10546000B7FC0122314B52421A8096E70121197094
:1054700005F0D2FFF5E70821307805F055FF637895
:10548000002B00D047E72C4B2D4F0293E388029A64
:1054900004211380294B307803932389039A1380C6
:1054A00063893B8006F078F9002800D033E7264B6B
:1054B0001B68002B00D12EE7039902983A880988CF
:1054C00000881B68984726E74379132B00D022E712
:1054D0000389012B0AD11D4B1B78022B06D1082111
:1054E000307805F021FFFFF72BFE14E7052000F0D0
:1054F00043FE08210200307806F056F80BE7C0465C
:10550000DE64FF1F05140000DD64FF1F7864FF1FC9
:10551000E842FF1FC942FF1FB264FF1F9364FF1FD1
:10552000B464FF1FB664FF1F8564FF1FC042FF1FE6
:105530008C64FF1F8E64FF1F8264FF1F8064FF1F47
:105540007E64FF1F8464FF1F7464FF1F7C64FF1F61
:105550008020C001014200D0E2E6CB0731D5324BBA
:105560001B78002B1DD0314E05AC3378052B1AD19A
:10557000023B23702E4B21001B7823722D4B1B788E
:1055800063722D4B187801F089FB002809D00720A1
:105590002A4B30701B68002B03D01B68002B00D0F7
:1055A00098470120BCE60E20254B06221B78254992
:1055B0002370254B1B78637002ABC01805F0ACFE5E
:1055C000D8E7022308001840194209D0174B1B786E
:1055D000052B03D11D4B188805F0FEFF02209FE626
:1055E0000424214203D0FFF737FD200098E608236A
:1055F00008001840194200D193E6154B1C78012C85
:1056000003D0022C0DD008208AE6124B124A13490F
:1056100013481B881288098800880094FFF7E0FD72
:10562000F1E7FFF78DFDEEE7B664FF1FDD64FF1FB6
:10563000C242FF1F9064FF1FDE64FF1F7864FF1FDC
:105640009264FF1FC342FF1F9164FF1FC042FF1FF0
:105650007C64FF1FB842FF1FBA42FF1FBC42FF1FFE
:10566000BE42FF1F10B502A804880B20002C10D1E9
:10567000496808784978090201430C48814209D1F8
:10568000022119800A4B59881170DB7800205BB227
:10569000537010BD074C0A20A142FAD10221198093
:1056A000034B998811705B79F0E7C0466E2A0000C1
:1056B0007C62FF1F6F2A0000F7B5150008AA168844
:1056C0004A680F4F14785278120222430A24BA42D1
:1056D00014D10122DBB2019200962A0005F024FDCC
:1056E000041E0BD1074B1B68002B07D068782A7863
:1056F0000002104342425041013098472000FEBD55
:1057000002290000F064FF1F30B501250379040071
:10571000BFB02B4225D01449408805F071F82842CB
:105720000CD0124B01A95B8D00220B8002234B8011
:105730000F4B5B888B80608802F042F90D496088CE
:1057400005F05EF8C0070CD50B4B01A91B880022A1
:105750000B8002234B80064B9B888B80608802F075
:105760002FF93FB030BDC046E864FF1FEC42FF1F79
:105770007C62FF1FE064FF1F4643FF1F10B5074C0C
:105780000749200004F0F2FF2000064904F0EEFF74
:105790000721054A054804F0ABFF10BDFFFF0000DC
:1057A000E864FF1FE064FF1F70B90011EC42FF1FA7
:1057B00010B5024802F086FF10BDC046095700111F
:1057C0000200F0B501270A480A4E51188B1A002B27
:1057D00000DCF0BD082415784308684038404000DC
:1057E000805B013C58406D08002CF5D10132EDE79B
:1057F000FFFF00008AB90011F0B500250F269D4279
:1058000000DBF0BD4C5D070944403440A400A058C3
:1058100001357840F3E70000F0B589B06A460D0025
:105820000B000F27110010351C78013326002409C6
:105830003E40167054700232AB42F5D12023024A2A
:10584000FFF7DAFF09B0F0BD90B90011F0B54E785E
:105850000B7889B036020C00170001901E43012A14
:1058600061D9954B9E4200D877E001339E421CD10E
:10587000062A17D1CA788B7812021A430B791B04B7
:1058800013434A7912061A438C4B5A6100221A704C
:105890005A808B4A5A608B4A9A608B4ADA600020A1
:1058A00009B0F0BD88225205EEE7884B9E423CD1FC
:1058B00082498B78002B00D0F6E00C2A31D10F22E0
:1058C000A3789343E278120213432279120413431C
:1058D0006279120613434B60E279A0791202024307
:1058E000207A00041043627A12060243CA60E27A08
:1058F000A07A1202024376484A81834208D80423E0
:105900006E49142201980B7005F006FD1420C7E7BC
:105910001201D21889235B059A42F0D801238B70BB
:10592000BDE7022AFAD00523EAE76A4A0123964234
:10593000E6D1FFF705FC052F0CD9E378A2781B020E
:105940001343227912041A4363791B061343624AF4
:105950000393136005F050FFA1E7584D2B78002BFF
:105960009DD1AB78002B00D1A0E02B8901339BB2F5
:105970000093B34200D091E0132AD4D9CF7C8B7C22
:105980003F02122120001F43FFF71AFF874200D079
:105990008EE0002E3DD1E378A2781B0213432279DA
:1059A000E96812041A4363791B06134303930A221E
:1059B0008B4212D1FF23A370E370237163716B8953
:1059C000002B09D1E37B227C1B0212041343A27B30
:1059D00013431B0901336B8100226B89002B8ED08E
:1059E000002A67D1686837013818000B6B6900031B
:1059F0000390984205D9686105F01EFFEB780133EA
:105A0000EB7068681022A11C381805F0DDFD2E81AE
:105A100045E76F89009A7B1E9BB293423AD1E278A8
:105A2000A37812021A43237905A81B041343627951
:105A30006C6812061A43EB6800920392211D0C2237
:105A4000049305F069FC0120260004A940421036A9
:105A5000FFF7E2FE013F012F17D1009A0B232861C7
:105A6000824200D04CE704221C49200005F0ACFD26
:105A7000042203A9686805F0B7FCE968039AFF23CC
:105A8000914200D13CE7F73B3AE73100FFF7C4FE13
:105A90001036DFE70923B742A4D831E7009BB342B1
:105AA00000D9FCE607232BE7022329E7032327E796
:105AB000062325E70A2323E7FFFE00006043FF1FBC
:105AC00000000111FFFF00005048593601FF00009F
:105AD000FFFF001102FF000034F000406C43FF1F85
:105AE00010B5034C0B000122210000F06BFA10BD31
:105AF000A15C00110B8870B506000D000224162B66
:105B000011D92B000322094900F05CFA041E0AD1C6
:105B1000074B2A881B88191C934200D9111C30009E
:105B200089B200F0EFFA200070BDC046CD5C0011D4
:105B30001A65FF1F10B54A780400013A0B000220D5
:105B4000012A07D80A78002A04D005222000024939
:105B500000F038FA10BDC046FB5C00110A7810B5A1
:105B60000B0004000220002A04D007222000024972
:105B700000F028FA10BDC046A75D00110A7810B5E4
:105B80000B0004000220002A04D009222000024950
:105B900000F018FA10BDC0460D5E001110B5034CA0
:105BA0000B000B22210000F00DFA10BD3D5E00112C
:105BB00010B5034C0B000D22210000F003FA10BDBC
:105BC000AF5E001110B5034C0B000F22210000F056
:105BD000F9F910BD095F00110A7810B50B00040037
:105BE0000220002A04D011222000024900F0EAF924
:105BF00010BDC046195F0011002310B51322190013
:105C000000F0E0F910BD000010B5034C0B001722A6
:105C1000210000F0D7F910BD6B5F0011002310B513
:105C20001922190000F0CEF910BD000010B5034C88
:105C30000B001B22210000F0C5F910BDA55F00116B
:105C4000F7B584890D0006000121002C22D0002325
:105C50008268D3561778002B1EDA0C2C1AD90C3C0C
:105C6000A4B2131940880093230002F086FE431E5D
:105C7000984101307B06DB0F6B703F23013C1F40D6
:105C8000A4B22870AF70AC80002C07D0B368013389
:105C9000AB6000210800FEBD0020EBE7AC60F8E738
:105CA0000B7803704B8843704B881B0A83700B7909
:105CB000C370042070470420022B06D100205378C3
:105CC00011781B02009A0B43138070470B880370F6
:105CD0000B881B0A437002207047042000998342FE
:105CE0000AD1537810781B0203430B80D378907845
:105CF0001B02034300204B807047F8B50D004B7822
:105D000001240021461C03702B788B4201D820000F
:105D1000F8BD6B78B01C4F1C012B10D1890069189D
:105D20004B88022233704B88B9001B0A73706918C4
:105D300005F0C2FC04360434A4B2F9B2E4E712233D
:105D400059436B185A88043132705B8810221B0A41
:105D50007370691805F0B0FC12361234ECE770B5B8
:105D6000049D14001E00052B01D8042070BD63782B
:105D700012781B0213432B80E378A2781B02134393
:105D800002226B802A71211D681D063E05F094FCDD
:105D9000B2B22A81E92AE8D82800A11D0A3005F00C
:105DA0008BFC0020E2E7002310B50A789A4201D864
:105DB000900010BD9A008A185488013304705488EA
:105DC000DBB2240A4470948884709288120AC270EC
:105DD0000430EAE710B51100029C062B04D0042021
:105DE0001022142B01D010BD022222714B780878AA
:105DF0001B0203432380CB7888781B020343638014
:105E00000431601D05F058FC0020ECE710B50C785B
:105E10008B7804315C43E4B203702200013005F05A
:105E20004BFC601C10BD0420022B06D100205378CF
:105E300011781B02009A0B431380704710B50C00B9
:105E40000A88023105F038FC208810BD70B50400C6
:105E50000D0004981100012B01D8042070BD1678A4
:105E600052781202324302800200F13255701470EF
:105E7000E125002C00D10C35023B9AB24280AA42A7
:105E8000EBD80231043005F017FC0020E6E70420CF
:105E9000009983420AD1537810781B0203430B8088
:105EA000D37890781B02034300204B80704710B5D5
:105EB0000C000A88023105F0FFFB208810BD0000AD
:105EC00070B501211E000420049C0E400B4218D125
:105ED000CB40DDB28D4214D90A49DBB20988994220
:105EE0000FD32300EE331D7033005800111849788A
:105EF000165C0902314301332152D9B28D42F4D8E4
:105F0000002070BD7843FF1F10B50C000A880231D5
:105F100005F0D2FB208810BD10B50C788B780431C9
:105F20005C43E4B203702200013005F0C5FB601C45
:105F300010BD10B511000298032B01D8042010BD2C
:105F400014785278043B120222430280CA788C787B
:105F50001202224342809AB28280EB2AEED80431A8
:105F6000063005F0A9FB0020E9E710B50C000B880E
:105F700003700B881B0A43704B8883704B881B0A85
:105F8000C3708A880430063105F096FBA08804307F
:105F900080B210BD0420012B03D100201378009A99
:105FA0001370704710B50C000B8803700B881B0A28
:105FB00043704A880230043105F07EFB608802306D
:105FC00080B210BDF0B589B003931E4B029242001F
:105FD0000700D05A019102F020F81325061E2DD09B
:105FE000029B01240370019B002B04D0001903992C
:105FF0009847001984B26B461B7A5BB2002B0FDA0C
:106000001021380002F01CFB1925002813D13000A4
:106010003219E1B202F066FC051E0CD10C34A4B2B8
:10602000042304AA380005A993800696948101F000
:10603000AFFD051E02D0300005F096FB280009B028
:10604000F0BDC0461865FF1F70B505000C000028A4
:106050000CD00020814209D010222000044905F014
:106060002BFB01202B7823736B78637370BDC046C4
:10607000D0B90011F0B506000D0017001C0085B066
:1060800002291BD00020102907D1022B07D0102B8A
:1060900003D115E00020102C08D005B0F0BD6946F2
:1060A0003800FFF7D1FF2A0069460BE0694630004F
:1060B000FFF7CAFF22006946380004E0022BE9D14D
:1060C0002A003900300005F057FAE6E7031CF028F3
:1060D00000D9F023032008499AB2013A0B80D31764
:1060E000034006499B189B100B80D30F04499B1853
:1060F0005B100B807047C0467C43FF1F7A43FF1F35
:106100007843FF1F034B1B888B4202D3024B400096
:10611000C15270477C43FF1F1865FF1F014B4000B1
:10612000185A70471865FF1F1722014B1A807047D5
:106130001865FF1F70B505000E2005F07DF9041EDF
:1061400013D0D023037000230622837007494570C3
:10615000033005F0B1FA064B2100DA8A62811B7E1A
:106160002373044B187805F04FF870BD3465FF1F9A
:106170002465FF1FCC43FF1F262803D8024B400095
:10618000C05A70470148FCE77E43FF1FFFFF000035
:1061900070B506000C00094D1C220021280005F0F6
:1061A0003BFA074B1E70074B1C7005F09DFA01234C
:1061B000002801D0002312202B7070BD2465FF1F22
:1061C000CC43FF1F4565FF1F70B505000D4C08004F
:1061D000E260A16010220021656005F0BDF9012890
:1061E00003D11021A06802F058FD102200212800E0
:1061F00005F0B2F9012803D11021606802F04DFDCD
:1062000070BDC0462465FF1F70B5041E05D100296E
:1062100003D006220D4805F04FFA0D4B1D78012DD5
:1062200011D1002C05D102221A7005F07DFA280048
:1062300070BD00221A70074B1B78FF2BF7D020008F
:10624000FFF778FFF3E70025F1E7C0463465FF1F4D
:106250002465FF1FCC43FF1F030010B5002801D1A8
:10626000002010BD00780B4A002803D15988D18244
:106270001B7913761378022BF2D10023984200D1B8
:1062800003331370044B1B78FF2B01D0FFF752FF31
:106290000120E6E72465FF1FCC43FF1F002911D032
:1062A00000280CD04B79012803D1402252421343DD
:1062B00003E03F221340032802D001204B717047B6
:1062C0004022F4E70800FAE770B5094D010028788C
:1062D00000280BD0074C0622200005F0EDF9210024
:1062E0002878FFF7DBFF200005F05EF870BDC046A0
:1062F0004465FF1F1E65FF1F00290AD0012808D131
:106300003F224B799343C02B03D0403B5A42534129
:10631000981C704770B5174D06002B78FF2B15D0D1
:106320000A2005F089F8041E10D0D0230370C83B62
:106330008370114B11491B784670C37006220430DC
:1063400005F0BAF92100287804F05EFF0C4B1B78A9
:10635000012B0DD10B4B1B68002B03D09B68002B2E
:1063600000D09847084B04211878084A05F04CF8EB
:1063700070BDC046CC43FF1F4465FF1F1E65FF1F55
:106380004065FF1F6C65FF1F7065FF1F60EA00001E
:10639000014B98687047C0462465FF1F014BDB68BE
:1063A000186870472465FF1F074B10B5DA6813683B
:1063B00001331360054B1878FF2803D08021C901F1
:1063C00005F02AF810BDC0462465FF1FCC43FF1F0F
:1063D000F7B50E0002F0C8F8051E1CD00E4B066281
:1063E0001F78002F00D10778AB791020019305F0BA
:1063F00023F8041E0FD0D0230380C73B8370019B7A
:10640000E91DC3700622043005F056F9210038005A
:10641000E66004F0F9FEF7BDCA43FF1F014B187890
:106420007047C0464465FF1F054B002805D1054B4A
:106430001A78054B002A00D1014B18007047C0465E
:106440003465FF1F4465FF1F1E65FF1F014B586821
:106450007047C0462465FF1F024B1868431E9841D1
:10646000C0B270474865FF1F421E03000120152A75
:1064700003D9FF3B5A425341D8B27047F0B51C00D4
:1064800000230E0085B0039002920B70029A934293
:1064900001D3002019E0E55C5A1CD2B2002DF8D0DF
:1064A000029851198142F4DC0233DFB2A35C180078
:1064B0000193FFF7D9FF002807D0013D019A039906
:1064C000EBB233708A4202D1E01905B0F0BDDB199E
:1064D000DBB2DBE710B50C0002F09EF803001220DF
:1064E000002B03D02100588804F02EFF10BD0000BF
:1064F00070B50E4D84006359002B15D0186A002822
:1065000001D005F019F92B59586A002801D005F07F
:1065100013F92B59986A002801D005F00DF9285974
:1065200005F00AF900232B5170BDC0465465FF1FCA
:106530001C4B70B504000E00150099420AD11A4B8D
:106540001B68002B01D1122070BD1B68002BFAD0F4
:106550009847F9E7154B994215D1134B1B68002B4F
:106560000AD01B68002B07D09847002804D1104B95
:106570001C70104B1D70E7E729002000FFF7AAFFF1
:106580000028E1D1F3E7080001F0EEFF0028DAD09F
:1065900003780320A342D7D12900300004F0D4FEB1
:1065A000D2E7C046FEFF00005065FF1FFFFF00005E
:1065B0004D65FF1F4C65FF1FF7B50400808801F093
:1065C000D3FF0025A84203D00578A08802F008F880
:1065D0001C4E3378002B1FD0AB421DD11A4B280024
:1065E0001978FFF777FF002818D000233370A379BC
:1065F0000820A778A688019304F01EFF011E0DD085
:10660000D0230370CA3B8370019B477086808371DF
:10661000280004F0F9FD01E0002DE8D1A0880B4B23
:106620008200D358002B01D0FFF762FF1721A0880A
:10663000FFF768FDA08801F027FDA08801F0FEFDAE
:10664000F7BDC0464D65FF1F4C65FF1F5465FF1F1A
:10665000F0B587B01D000CAB1B88070001930DAB94
:106660001B88142002930EAB1B88160003930FABFC
:106670001B880091049310AB1B88059304F0DCFE8B
:10668000041E1AD0D0230370CB3B47708370C670B2
:10669000062229000430002D11D005F00DF8019BD1
:1066A00021006381029B0098A381039BE381049BEB
:1066B0002382059BA37404F0A7FD07B0F0BD04F08E
:1066C000ABFFECE7F7B5009308AB1B8807000C2085
:1066D0000D001600019304F0AFFE041E13D0280035
:1066E00001F042FF00280FD00078D0232370C93B6F
:1066F000A370009B21002381019B6770A580E68029
:10670000638104F081FDF7BD014B1878EDE7C046C9
:10671000CC43FF1F13B5040064890389C2888188B4
:10672000C0780094FFF7CEFF13BD000010B5044CF5
:106730002068002803D004F0FFFF0023236010BD71
:106740005865FF1FA122F0B5818892004A43384B5B
:10675000384F1B6804009B189D2292009B18827979
:1067600089B01A603B68002B5FD01D78324B1B68E4
:10677000002B04D05B68002B01D000209847260036
:1067800008363100E079FFF7B7FD237DE0710200A4
:10679000E0780493638A29000393238A0293E389B0
:1067A0000193A38800933300FFF752FFE378002B97
:1067B0000BD1E289A379A18802920196E27928009F
:1067C0000092012201F0DAFEE0703B68002B20D03D
:1067D000FFF7ACFF194D287800281AD0184B19780C
:1067E000FFF778FE002814D02B78E678082007936E
:1067F000A78804F021FE011E09D0D0230370CA3BF4
:106800004670837087808671079804F0FDFC002332
:106810002B701721A088FFF775FCA08801F034FCCD
:10682000A08801F00BFD09B0F0BD064B9DE7C04606
:106830003409FF1F5865FF1F6C65FF1F4D65FF1F63
:106840004C65FF1FCC43FF1FF8B5070008000E0082
:1068500001F08AFE041E18D02620FFF78DFC051ECD
:1068600000D12578062004F0E7FD041E0DD000219C
:10687000062204F0D1FED0232370C23B21006770B2
:10688000A370A680E8B204F0BFFCF8BDF0B585B0F7
:1068900001930AAB1B78070002930BAB1B7808002F
:1068A0000D000092039301F05FFE061E22D010201F
:1068B00004F0C2FD041E1DD01022002104F0ACFE25
:1068C0002620FFF759FC002800D13078D023237010
:1068D000C13BA370009B21002372019B6770637210
:1068E000029BA580A372039BC0B2E3720C9BE36082
:1068F00004F08AFC05B0F0BDF7B50D00019001F081
:1069000033FE071E20D00E2004F096FD041E1BD07F
:106910002620FFF731FC061E00D13E78D0232380CD
:10692000C53B0622A370F91DE01C04F0C5FE019BC7
:106930002A0063810123DD401A401D40210022739B
:106940006573F0B204F060FCF7BD0000F0B585B0EF
:10695000029010000D0017000A9E039301F004FE40
:10696000041E31D0029B002B2ED1039B02795B07C2
:1069700024D5122313430422002E08D10B99002999
:1069800005D10C99002902D10D9900291AD01A437A
:106990000D9B2271002B00D0C9E0002E00D1CFE06A
:1069A000002D00D0CCE0606A002801D004F0C4FEC5
:1069B0001C21300004F058FE606205E002239A4377
:1069C0000E33D7E793432371654BBA00D458002C9C
:1069D00000D1AAE0002E10D0236A002B03D11C2086
:1069E00004F05AFD20625E4BBA00D358186A0028A2
:1069F00003D01C22310004F05FFE0C9B002B12D050
:106A0000574CBB001D596B6A002B03D1162004F0B4
:106A100043FD6862BB00E358586A002803D0162281
:106A20000C9904F049FE0D9B002B11D04C4DBC007D
:106A30006659B36A002B03D1142004F02DFDB06217
:106A40002B59986A002803D014220D9904F034FEC3
:106A5000380001F089FD051E67D0414BBA00D358BC
:106A6000002B62D01A6A3420002A00D11C389A6A9E
:106A7000002A01D0143080B20B9A002A01D01C30B9
:106A800080B25B6A002B01D0163080B204F0D4FCD7
:106A9000041E4AD01822002104F0BEFD2620FFF774
:106AA0006BFB0190002801D12B780193D023237038
:106AB000029B200063700A23294EA370039BBD0034
:106AC000A371AB59A780196A1830002905D01C2280
:106AD000A06004F0F1FD200034307359996A002958
:106AE00007D0030014221433E060029304F0E4FDA5
:106AF00002980B9B002B08D003001C221C330B991F
:106B00002061029304F0D8FD02987359596A002954
:106B100003D01622606104F0CFFD6B462100187986
:106B200004F072FB3800FFF7E3FC05B0F0BD102263
:106B30000D9B0D991B69A018236204F0BDFD2CE785
:106B40000B9B002B00D13FE7012D00D03CE7606A92
:106B5000002801D004F0F0FD1C210B982AE7C04664
:106B60005465FF1F10B5044C2068002803D004F0C2
:106B7000E3FD0023236010BD4865FF1F0B4B07B5E5
:106B80001A68002A01D100200EBD6946531C01205D
:106B900012780731FFF772FC0028F4D00278012345
:106BA000100018401A42EED0EEE7C0466465FF1FA1
:106BB000F0B51F4F01203B6887B0002B25D09B7894
:106BC000059300F0B3FB002821D00A20FFF7D4FA88
:106BD00004000B20FFF7D0FA164B05001E78731E39
:106BE0009E413B68F6B2191DD878FFF757FB3B680A
:106BF0002900DA7A043303929A7901930292009081
:106C000033002000059A04F087FD07B0F0BDFFF7C0
:106C1000B5FF002805D00620FFF7AEFA04000720D4
:106C2000D8E70820FFF7A8FA04000920D2E7C046F9
:106C30004865FF1F4465FF1F70B50A4E0400337896
:106C40000D00FF2B0DD0042004F0F6FB011E08D030
:106C5000D0230370CE3B45708370C470307804F04D
:106C6000D3FA70BDDC43FF1F70B5040006200D0091
:106C700004F0E2FB011E0AD0D0230370CD3B8370E9
:106C8000054B44701B688580187804F0BDFA002C11
:106C900001D0FFF767FF70BD4865FF1FF8B5264FAD
:106CA00006003B680D001124002B05D10522234B63
:106CB0001B78134202D112242000F8BD204A102470
:106CC0001268002AF8D01278002AF5D0DB0719D50F
:106CD0002B789A1E012A1AD80C2004F0DDFB13240D
:106CE00038600028E8D000230A224370290006708B
:106CF000023004F0E1FCFFF75BFF041E0AD0FFF74F
:106D000031FFD9E700F012FB0028E1D1E4E7002BC6
:106D1000E2D0D0E70B4B1B78032BCDD11D20FFF722
:106D20002BFA094B18800028C6D0084B042118788C
:106D3000074A04F069FBBFE74865FF1F4565FF1F71
:106D40006465FF1F4465FF1F4265FF1F7065FF1FDD
:106D500060EA0000F7B50193194B14001A78052377
:106D600006000F0012201A4221D0012920D1154B14
:106D70001D68002D1BD002201F2C18D8002C02D01B
:106D8000019B002B13D0104B1F221E706E1C002184
:106D9000300004F041FC01992200300004F08CFC2A
:106DA000310020002C70002F06D004F085FAFEBDC3
:106DB000064B12201D68DCE704F076FBF7E7C046BF
:106DC0004565FF1F6465FF1FDC43FF1F6065FF1FF4
:106DD000F8B50F4E12243368002B17D01B780F3CE8
:106DE000834213D100250B4F0221387804F09CFA1E
:106DF000094B042138781D8004F096FA074B2800CF
:106E00001D8033685C7004F03FFC04002000F8BD76
:106E10004865FF1F7065FF1F5C65FF1F4265FF1F10
:106E200070B5012823D11B4C2388002B03D01A4AAC
:106E30001578002D07D0194B1B68002B02D018784D
:106E4000FFF7C6FF70BD3B2B02D93C3B2380F9E71F
:106E5000134E0221307804F067FAFA222388920058
:106E600002215A43307804F09FFB2580EAE70B4B60
:106E70001B68002BE6D00B4B1B785B07E2D5084B59
:106E80000221187804F050FA0022024B1A80FFF712
:106E900069FED7E75C65FF1F4065FF1F4865FF1F60
:106EA0007065FF1F4565FF1FF8B51E4D2868002857
:106EB00003D004F041FC00232B601B4E30680028F7
:106EC00003D004F039FC00233360184F05243B78CD
:106ED00018002040234221D0154800F02BFA3B78BF
:106EE000234213D0202004F0D7FA2860002813D0C2
:106EF0002022002104F090FB202004F0CDFA041E93
:106F0000306005D02022002104F086FB002004E040
:106F1000286804F011FC2C601320F8BD00F00AFA78
:106F2000F4E7C0466465FF1F6065FF1F4565FF1FEE
:106F3000D043FF1F10B50A4C23681A1E0ED000283C
:106F400008D10130587004F09FFB002805D0236859
:106F5000002B02D00021FFF787FE0122100010BD98
:106F60004865FF1FF7B5274E050033680191181ECD
:106F700021D05C78244F012C30D1FFF7FFFD002891
:106F800025D02000FFF7F8F80400412814D91F4B42
:106F9000022118781E4A04F037FA1E4B3C3C1C8034
:106FA000022233685A703B78002B14D128000199D3
:106FB000FFF75AFE0120FEBDFA2292004243002A4A
:106FC000EED0124B0221187804F0EEFAE8E7FFF752
:106FD000D3F80200F3E700233B70EBE73B78002B8C
:106FE000E8D1032004F028FA011E08D0D023037052
:106FF000CC3B457083703368187804F005F9FFF7CF
:10700000B1FDD7E74865FF1F4065FF1F7065FF1F93
:1070100060EA00005C65FF1F10B517498388020015
:107020008B4220D011D815498B4217D0144900202B
:107030005B1899B2012907D8926811785A425341D6
:10704000D8B2FFF7F9FD012010BD0E4A00209B18B1
:1070500007229BB29A424041C0B2F5E78368187894
:10706000FFF768FFF0E7836899785A780902187883
:107070001143FFF777FFE7E70A2000000620000032
:10708000F8DFFFFFAFDFFFFF014B18707047C0460E
:10709000DD43FF1F10B5064C207001F041FA207847
:1070A00004F0FAF80521207800F062FD10BDC0461A
:1070B0007065FF1F0BB273B50D00002B00DBC4E041
:1070C000884B187804F088FB041E0ED00378912BAF
:1070D0000FD0A22B00D1A1E0834B1878FF2852D00B
:1070E000210004F091F800284DD180200002684072
:1070F00076BD43780F2B76D013D8052B70D00E2B8E
:10710000EAD18088794B98422BD8794B98421BD88A
:10711000784B9842E0D1A3681878591CFFF774F8AF
:1071200038E03E2BD8D18378032B74D06CD8012B58
:107130006ED0022BD0D1704B1B68002B23D05B6824
:10714000002B20D098471EE06C4BC0180C28C3D8E9
:1071500004F09AF81DC2C2150BC20B0B0B3223C2EE
:107160003C00674BC0180728B6D8664B1B68002B3D
:1071700009D01B68002B06D0200098470AE0A368BE
:107180001878FFF7C7F8200004F0D6F9ADE7A0683B
:10719000FFF762F800289FD0F5E7A3681B78002B63
:1071A000F1D0554B1B68002BEDD01B68002BEAD0AB
:1071B000210055489847EDE74F4B1B68002BE2D064
:1071C0001B68002BDFD021005048F3E7504B1B68B1
:1071D000002BD8D05B68002BD5D021004348E9E7CD
:1071E000FFF7EAF9CFE780884A4B984203D04A4B31
:1071F000984200D070E7464B1B68002BC3D05B68F9
:10720000002BC0D02100D5E7153B012BBBD963E78C
:10721000FFF798FAB7E7FFF77DFAB4E73F4B1B7823
:10722000042B07D100236A4613800179408800F0BF
:10723000C5FCA8E7364B1B68002BA4D05B68002B6D
:10724000A1D00100364898479DE7012421420AD089
:10725000294B1B68002B04D05B68002B01D0002059
:107260009847012043E78B070AD5264B1B68002B64
:1072700004D05B68002B01D020009847022036E73D
:107280000421280008400D4200D131E7254E338803
:10729000002B21D0013B9BB23380002B1AD1FFF78A
:1072A000DBF800280AD0204B1C70164B1B68002B03
:1072B00004D05B68002B01D020009847FFF7C6F888
:1072C000694601F001FD6846FEF7FEFF1D20FEF74E
:1072D00053FF308004200AE7024B187804F024F8AA
:1072E000F8E7C0467065FF1FDD43FF1F0E2000005A
:1072F00001200000091000006865FF1FFEDFFFFF8E
:10730000AFDFFFFF6C65FF1F0C2000000B200000AB
:107310005065FF1F0D200000132000004565FF1F72
:10732000FFFF00004265FF1F4065FF1F10B501F021
:107330009BF910BD014B18607047C0466C65FF1F7C
:107340000B880020162B01D817230420014A138034
:107350007047C0461A65FF1F00207047074A0300A8
:107360001188814207D091880020994202D10130D2
:107370008000101870470020FAE7C0467865FF1FAC
:10738000F0B58F7806000D00C5B01E2F15D1FFF7A0
:10739000E5FF051E03D10024200045B0F0BD00220A
:1073A0003B003100C078009200F0B2FB0400A81C42
:1073B00000F0D2FBFF23EB70EEE7264B062403938D
:1073C0001B78FF2BE8D0182FE6D87B08224A013B18
:1073D000DB0002929A589446002ADDD0029AD31814
:1073E0005B68002BD8D00878002802D14B78012B9D
:1073F00002D10624122FCFD107AFAB88697800974E
:107400006446AA68A047041EC6D1AB78029A5B08FE
:10741000013BDB00D318390030005B689847041E3D
:107420000BD1AB78042BB6D0039A31001078220030
:10743000009700F06DFB0400AEE76A78002AABD13C
:10744000AA7805A93B88087130000A704B80FEF7C6
:1074500047FBA0E7E043FF1FE0B900111D4B37B524
:10746000050098420BD000290AD1FFF777FF0028CA
:1074700005D11948FFF772FF002800D0058037BDFD
:1074800001291AD1FFF76AFF041EF8D001235B42DD
:107490000380A378FF2BF2D0FE2B07D00023E078E7
:1074A0001422009329001E3300F032FBA01C00F0D0
:1074B00053FB01235B426380E1E70229DFD10139FD
:1074C00001F0BEF80028DAD12800FFF747FF041EBC
:1074D000DFD1D4E7FEFF0000FFFF0000022210B55D
:1074E000074B52421A80074801325A809A80DA804C
:1074F00000F07EFA044801F025F8002010BDC046D7
:107500007865FF1F817300115D7400110388F7B562
:107510000400002B02D102252800FEBD4268022192
:10752000137825485268FEF7A5FD00282ED0234F7A
:1075300001253A88002AEFD0802321885B020125AB
:107540009B1A9942E8DC0C2003F0A6FF061E31D0FE
:107550003B8822889C4600231800019561469DB215
:10756000491989B2AA421BD8002801D062443A8046
:1075700000233000082208C0210004F09DF8104AC2
:107580001368002B13D100251660C5E7626802213D
:1075900013780C485268FEF76DFD0028C7D1BAE792
:1075A00060681D014019418101330198D6E71A0036
:1075B0001B68E6E71325AFE74EBA0011DE43FF1F55
:1075C0007465FF1F4CBA0011014B18707047C0461C
:1075D000E043FF1F14230A0010B51A40194204D0DB
:1075E0000122102101F048F810BD4B06F9D401200A
:1075F00088434000F8E710B514008B0604D501223B
:10760000102101F039F810BD08230A001A40194270
:1076100002D14BB2002B0FDA102101F02DF8002817
:1076200008D02300F2331B78002BECD0F134237800
:10763000012BE8D10020E6E703208907FAD4E2E72E
:10764000F0B51F00184B85B01C68019002910392A1
:10765000002C27D1200005B0F0BDA5683301ED183E
:107660006B89019A934211D3029A93420ED8002F4C
:1076700004D10A9B002B10D12C00EBE73B002978AA
:10768000039A6868FEF7F6FC0028F2D10136B6B21C
:10769000A388B342E1D82468DAE7A3680A9A5B8931
:1076A0001380E9E70026F3E77465FF1F37B50C0088
:1076B0000A8849880123914217D3002A15D0651DF5
:1076C00023792A0002210A48FEF7D4FC102300285F
:1076D0000BD023796188208800242A000094FFF7CA
:1076E000AFFF0A23A04200D0230018003EBDC046D1
:1076F0004EBA001113B50A00088849880123884250
:107700000BD8002809D00024137905320094FFF724
:1077100097FF0A23A04200D02300180016BD13B51E
:107720000A0008884988012388420BD8002809D01C
:107730000024137905320094FFF782FF0A23A04248
:1077400000D02300180016BDF0B58BB003904A8816
:1077500008880E000123824255D3002853D000230D
:10776000012704AC23700022718813000092FFF7F8
:1077700067FF051E3ED02078002835D12B78022BDC
:1077800018D167706A8983000130E31880005A803D
:1077900069680222201803F08FFF23780133DBB2DF
:1077A0002370042B19D93B006889013080B2002B6B
:1077B000D9D01FE002236370122358436A8923182B
:1077C00004305A8069681022201803F075FF23786E
:1077D0000133DBB22370002BE5D10C4A6B899B1877
:1077E0005A425341DBB2DFE76378012BE4D12B78B7
:1077F000022BC7D022780A23002A04D02100039844
:10780000FEF798F9002318000BB0F0BD0100FFFF50
:107810000F4BF0B504001868002816D083685D8906
:10782000A54207D88288AE18B44203DA12019A182A
:10783000934201D10068EFE71E005F891036A7422E
:1078400004D1002900D00D801800F0BD3300EFE70F
:107850007465FF1F70B505000C0008880021FFF754
:10786000D7FF03000120002B04D022002800197A42
:10787000FFF7C1FE70BDF7B50C0000250190230095
:10788000EE331B78AB4201D800200AE06B00E65AC9
:1078900000213000E718FFF7BBFF002802D1268047
:1078A0000130FEBD017A0198FFF794FE002802D056
:1078B0003B882380F5E70135EDB2E0E710B5040021
:1078C00008880021FFF7A4FF03000120002B03D04C
:1078D0002000197AFFF77EFE10BD0000054B1B68E3
:1078E000002B01D1180004E09A6852898242F6D137
:1078F000988870477465FF1FF0B50E27002687B083
:10790000039302ABFF183E8005001F4B4089140013
:10791000984207D02B78013000976A6880B2FFF751
:107920008FFE060002212B7818486A68FEF7A2FB3A
:1079300000280FD06C892000FFF7D0FF002802D06C
:10794000013C0419A4B2039B002B00D01C80300022
:1079500007B0F0BD02212B780D486A68FEF78AFB5C
:107960000028E7D102212B780A486A68FEF782FBDB
:10797000002807D0002EDED03B88A342DBD17489DB
:10798000013CDFE76C89DEE7FFFF00004EBA001123
:107990004CBA00114ABA001110B50C00FFF7DEFC1A
:1079A00003000220002B0AD0002C00D023609B781B
:1079B0001720FE2B03D00138FF2B00D1002010BD73
:1079C00073B50D0001A904001600FFF7E5FF1728A5
:1079D00005D0002E04D129002000FEF727F976BD3E
:1079E00001221021200000F047FE0028F3D0F6E726
:1079F000014B18607047C0468465FF1F37B56B4662
:107A00009D1D010004000222280003F085FC2B8844
:107A1000B02B0ED12379122B09D12300FA331B7816
:107A2000012B06D10121608800F0E0F801E01B2B5A
:107A3000F8D037BD10B5054B0421187000F098F848
:107A4000FFF74CFDFEF770FB10BDC0468865FF1FB9
:107A50000020F0B50BB20F0087B0834234DA274B19
:107A6000187803F0B9FE051E2BD00378A02B25D182
:107A700003AE3100FEF7E4F8041E0BD1B378DB0748
:107A800024D51F4B06341B68002B03D031006888B7
:107A900098470400A868002801D003F065FE002C78
:107AA00008D1184A039B1340174A934206D0B37873
:107AB0001B2B03D00121688800F098F8280003F000
:107AC0003BFD80200002784007B0F0BD0F4B1B68E3
:107AD000002B10D0310068889847041EDAD07378E4
:107AE000002BD7D1B27801A90A704B800C7168883D
:107AF000FDF7F6FFCEE70624F1E7C0468865FF1FD5
:107B00008065FF1F00FFFF00000112008465FF1F5A
:107B1000F7B50190FC200D0017001E0003F08CFC4F
:107B200004001320002C12D0B02320002370089BE7
:107B3000F4226770658026710830002B08D0190088
:107B400003F0BAFD2100019803F05EFB0020FEBDAA
:107B5000089903F061FDF5E710B5041E06D0007822
:107B6000FD2803D803F050FEFF23237010BD000052
:107B70000A1F93B210B504000220032B05D88240DF
:107B80000020024BD1529B189C7010BDA865FF1FAE
:107B90000B8870B5043B04000D000220032B0BD8AA
:107BA0000121200000F04CFD03001420002B03D025
:107BB0002900200000F0DEFB70BD000007B51300B7
:107BC000034A00920A00012100F02CFC0EBDC046C1
:107BD000F97D001107B5019203220092024B0A00C1
:107BE000122100F049FC0EBD777E001107B56B46EF
:107BF00001AA11800449D88008780633012802D1EF
:107C0000190003F0B1FB07BD8965FF1F0C4B10B5D0
:107C100018700023FF210B4A1380138193819380F6
:107C2000094A53801370517293819372D174D38235
:107C30001375517703F0C0FC00F0FCF910BDC0468D
:107C4000B865FF1FA865FF1F8A65FF1FF0B58DB0DF
:107C50006B46002003910C229B5E834200DBB0E068
:107C60005D4B187803F0B8FD051E00D1A4E0037841
:107C7000902B00D09DE006AF01004688380000F050
:107C800013FA79680400002900D19CE03B88052B99
:107C90006ED13B89032B1CD905AC200000F0A2F863
:107CA0006288172A61D83989131D994231D17968C0
:107CB000237804310291D90738D5607800F08EF925
:107CC000071E06D0002303712378012B08D0132B45
:107CD00023D0A868002800D178E003F045FD75E0C6
:107CE0006288029909A800F0A6F80290380000F016
:107CF0008BF909AA2378387A019200223100009288
:107D0000029A00F012F9380000F064F9029B002B8F
:107D1000DFD0300000F080F9DBE70378032BD8D107
:107D20006288029909A800F0D6F8DEE7122B13D179
:107D3000029909A800F0B5F8021EEAD127498B88FC
:107D4000002BC6D0887909A9237801916178009128
:107D5000310000F0EAF8BCE7002302AA9383300068
:107D6000617809AAFFF72AFFB3E71D4B0993F6E7ED
:107D7000042B02D09A1F012AABD8184A043B9B005F
:107D8000995A0029A5D0D218907831003A0000F015
:107D9000AEF800289DD13B88042B03D00121300090
:107DA000FFF724FF012C04D1A868002801D003F0BC
:107DB000DBFC280003F0C0FB8020039B0002434053
:107DC00018000DB0F0BD012800D182E7012130007C
:107DD000FFF70CFFEDE7C046B865FF1FA865FF1F62
:107DE000010017000B7803704B784370CB788A78CA
:107DF0001B021343438070470A88030002700A88FD
:107E0000120A42700A88012A06D14A8882704A887A
:107E1000120AC2700420704702208242FBD14A88B5
:107E200004309A704A88120ADA708A881A718A882D
:107E3000120A5A71EFE710B50400012082420CD9F2
:107E40004B780A781B0213432380834206D1CB78F8
:107E50008A781B0213436380002010BD022BFBD1E4
:107E6000CB788A781B02134363804B790A791B0213
:107E70001343A380F0E70B8803700B881B0A437041
:107E80004B8883704B881B0AC3708B8803718B8867
:107E90001B0A4371CB888371CB881B0AC3710820EE
:107EA000704703000120082A14D14A78087812028A
:107EB00002431A80CA788878120202435A804A79AB
:107EC0000879120202439A80CA7988791202024321
:107ED0000020DA80704710B504000120022A05D185
:107EE00000204B780A781B021343238010BDF8B59D
:107EF000060010200F00150003F09EFA0400012078
:107F0000002C0ED0A0230C22290023806780201D86
:107F1000002D07D003F0D0FB2100300003F074F9EE
:107F20000020F8BD03F078FBF6E7F7B51E000090DF
:107F300008AB142017001D78019103F07DFA041E90
:107F400012D0A2230370019B47704380099B0571E7
:107F500046710C220830002B07D0190003F0ACFB4F
:107F60002100009803F050F9F7BD099903F054FB84
:107F7000F6E737B5041E0FD04388002B0CD0002540
:107F8000C1881323007A172201950095FFF7CDFFD2
:107F9000FF2365806372257037BD000010B50C4962
:107FA00004004A88002A09D08B89002B05D00020C4
:107FB000CB8A0222834201D010BD012213000A2085
:107FC000434300204032C854C81842800472F3E78B
:107FD0008A65FF1F0023438003707047094B00210F
:107FE0001A0010B55C88002C06D01C79844203D19D
:107FF0000A234B43D01810BD01310A330329F1D1B4
:108000000020F8E78A65FF1F10B50400407A03F0EE
:10801000FBFBFF23637210BD7047043010B580B2C4
:1080200003F0AAFB002803D00421494203F05CF9C5
:1080300010BD000070B50025104CA0682580A581FA
:10804000A580A84202D003F08FFBA56000250C4C50
:108050000C4B606D1D80230058331D70A84202D068
:1080600003F082FB656500256068002801D003F0FD
:108070007BFB013508340A2DF6D170BD5066FF1F19
:10808000F465FF1F4466FF1F70B5041E09D1054D3E
:108090002880A881A880A868002802D003F064FB8B
:1080A000AC6070BD5066FF1FF0B54B8885B0019382
:1080B000002343600A7905000F00022A00D07BE00C
:1080C000CA88032A17D98B685E7819783602DC785B
:1080D000D8790E4399781B7A24021B020C43034380
:1080E00053495BBA0B80331D93421ED1042C04D03C
:1080F000631F022B0ED9012015E0019A4D4B12018E
:10810000D35A002B06D00198FFF7BEFF4A4A1369E5
:10811000013313610421B8682E812C80494203F099
:10812000E3F86860002005B0F0BD434D042C06D094
:10813000631F022B0FD9EB680133EB60DBE7019A79
:108140003C4B1201D35A002B05D00198FFF79CFF3E
:108150002B6901332B61374B30000293019B029A4C
:108160001B010193002301998C468B521300634439
:108170009C8003939E81FFF750FF039B041E986031
:1081800016D00421B868494203F0AEF8FA8801001D
:10819000043A200003F090FA0199029AFB888A5A67
:1081A000043B9B18029A8B522B6801332B60A2E789
:1081B000AB690133AB619EE71E4B0293019B1E012D
:1081C000029BF35A002B2DD002998C19A06800282D
:1081D00028D0012A26D1FA889B189BB27352A18914
:1081E000994217D39B1AC018B96803F065FA029B2D
:1081F000A289F35A934200D07DE700222B81A38805
:108200002B80A3686B60029BF2520B4A53680133C8
:10821000536070E7084A9368013393600198FFF751
:1082200033FF68E7044A536901335361F6E7C046F8
:10823000BA65FF1F5066FF1FC065FF1F70B5051EA2
:1082400015D10B4C0B4B1880230058331870606D00
:10825000002802D003F088FA656525005035606873
:10826000002801D003F080FA0834AC42F7D170BD89
:10827000F465FF1F4466FF1FF0B51700A12285B00B
:10828000920001934243394B06001B680C009B1877
:10829000D933FF331D78FDF741FF0430854204DDFB
:1082A0003000FDF73BFF0430C5B2BD4207D33A00B2
:1082B00000213000019B03F087FA05B0F0BD2900D2
:1082C000380003F009F82300C6B250331E70039340
:1082D000019B29006365380002F0F6FFCBB20293E0
:1082E000002B02D0039B01361E7000262300503362
:1082F00003931B78B34204D8606D002831D100206D
:10830000DBE7029A2800002A04D0013B1000B342A8
:1083100000D02800F700E719387003F055F87860AE
:1083200000280ED03A78019903F0C6F9019A3B78FB
:108330000136D3180E4A0193D369F6B20133D361E3
:10834000D4E7039B18706065A74205D1084A132043
:10835000D36A0133D362B0E7606803F005FA0834EA
:10836000F2E703F001FA00236365C8E73409FF1F51
:10837000C065FF1FF7B50D0007000421686802F013
:10838000B3FF2B89040003702B891B0A43702B88D1
:1083900083702B881B0AC3702E8902250436F6B21F
:1083A000F42E15D81B4B9F4214D10C2003F044F837
:1083B0001135011E0CD0902303708E3B0371043BDA
:1083C0004380154B8460C680187802F01DFF00259D
:1083D0002800FEBD5C237B43104AD318009358331A
:1083E00001931B78002B0FD1030032003800009955
:1083F000FFF742FF019B05001B78002BE8D13800F6
:10840000009903F041F8E3E7054A0725536A013371
:108410005362DDE7FEFF0000B865FF1FF465FF1F34
:10842000C065FF1FF0B587B0009017200F00160041
:108430000193FFF7F2FD1325041E19D00C98031EBB
:1084400002D00199201D9847030AE370052302AA70
:10845000A0700430908127700098667003A9938003
:108460000494FFF787FF051E02D0200003F07CF97B
:10847000280007B0F0BD0000F0B587B01F000CABBE
:108480001B780391059301210DAB06001C78049223
:1084900000F0D6F81425002821D02000FFF77EFD3B
:1084A0000135041E1BD01149059B0A780370013267
:1084B000D2B2131EC68001D101231A000B702271A3
:1084C0003000049B03990097FFF7ACFF051E09D10C
:1084D000230021000648074A093303F0B5F82800B5
:1084E00007B0F0BD002363802370F8E7BC65FF1F71
:1084F000737F001130750000F8B505000E00064CC2
:10850000064F2368002B02D031002800984704341E
:10851000BC42F6D1F8BDC0466066FF1F7466FF1FFF
:108520000123064A5B425380002313715362044ABD
:10853000136053609360D360136170477466FF1FCC
:108540006066FF1F0200002310B506499C00085911
:10855000002801D1625010BD0133052BF6D1132044
:10856000F9E7C0466066FF1F034A5388181A434262
:1085700058414042104070477466FF1FF0B585B007
:1085800002930AAB1F780CAB1B88009008000E000A
:1085900001920393FFF7E8FF05001120002D1BD186
:1085A0000E48FFF7E1FF04001520002C14D006222E
:1085B0000B99A771E01D03F07FF8019B3000237138
:1085C000029B29006371009B66802370039B656298
:1085D000E381FFF791FF280005B0F0BDFFFF000029
:1085E00010B5FFF7C1FF04000220002C12D06088F4
:1085F0000121FFF781FF606A002801D003F09CF899
:1086000028220021200003F007F8012300205B420C
:108610006380207110BD000030B5074A074C5588B3
:10862000010013780020A54204D05B1A59424B4147
:108630005842104030BDC0467466FF1FFFFF000067
:10864000084A10B501230C00904208D0FFF78CFFB8
:10865000031E04D0037923405A1E9341DBB2180055
:1086600010BDC046FEFF0000024B1879431E984122
:10867000C0B270477466FF1F70B504000D0016008D
:10868000FFF772FF002804D10D4B9C4200D014303C
:1086900070BD416A03790520002907D012221A40D3
:1086A000102A02D10520002EF2D10F20DB06EFD5D3
:1086B000897E0C20A9428941494249420840E7E7A6
:1086C000FEFF0000030010B5002800D110BD0348D4
:1086D000034A41889142F9D09847F7E77466FF1F33
:1086E000FFFF0000002330B5C45CCD5C6C40D45467
:1086F0000133102BF8D130BD0F23002210B5C45C1C
:1087000064002243CA54C25CD209013BF7D210BDB7
:108710000200010010B52032103102F005FF10BD3B
:10872000F0B58BB00390102005931700049102F070
:10873000B3FE0090102002F0AFFE009B13240190C6
:10874000002B05D000280CD11324009802F0F4FF70
:10875000019B002B02D0180002F0EEFF20000BB0AE
:10876000F0BD102002F098FE0600102002F094FEEA
:1087700013240500002E00D1AEE0002819D01022ED
:10878000002102F049FF32002900039802F0CCFEDC
:10879000041E0ED133787F2B51D830000099FFF79B
:1087A000ABFF009B1B787F2B53D801990098FFF7F4
:1087B000A3FF300002F0C0FF002D02D0280002F01D
:1087C000BBFF002CC1D1102002F066FE0600102075
:1087D00002F062FE0290002E7CD0002878D03A0091
:1087E0000F3223000125121105D00F333B4015B283
:1087F0005A4253411BB26A1E1201002B33D0049B14
:10880000D2B298180099029AFFF76CFF013D10222E
:108810000021300002F000FFADB2049F2D017D1950
:10882000AF4242D0002C33D0300002F085FF029BD3
:10883000002B00D189E7180002F07EFF85E72900B0
:108840003000FFF759FF28002549009AFFF74AFF3B
:10885000A7E729000098FFF74FFF28002049019A59
:10886000FFF740FFA5E70F210F4004998A18D9B2FE
:108870008F4208D9D15C06A819540133102BF6D1C8
:10888000029A0199C0E7791A48424141C901F2E7C9
:108890003900300006AAFFF725FF3200039806A929
:1088A00002F042FE10370400BAE7002CBCD13000C1
:1088B000029906AAFFF716FF320006A9039802F0F4
:1088C00033FE082204003100059802F0F5FEABE704
:1088D0001324A9E71324AAE7002800D06EE733E7A2
:1088E00054BA0011F0B58BB00F00160002250090AD
:1088F00000283FD0002A3DD00B1DDBB218000293A8
:1089000002F0CAFD1135041E34D0FDF747FD050005
:108910003A000099201D02F0AFFEEBB20393E37022
:108920002B0CDBB22F0A00936370FFB22B0E237067
:10893000A7700193FDF72CFD1022010006A802F09C
:108940009BFE2100029A04AB06A8FFF7E9FE051E74
:108950000DD1039B08223370009B04A9B370019BC7
:108960007770F370301D02F087FEFDF71DFD2000CB
:1089700002F0E2FE28000BB0F0BDF0B58FB00D00A4
:10898000149E039004920593002A03D10224200030
:108990000FB0F0BD002EF9D00398FFF7E5FD1424C9
:1089A000071EF4D07278337812021A43B3781B048E
:1089B0001343F27812061A43036A0192934201D3D9
:1089C0000133E3D1002D03D03B7901249B07DED591
:1089D0000822002106A802F01FFE059B1324043381
:1089E000DBB21800029302F057FD051ECFD0059AA6
:1089F0000499043002F040FE04223100280002F005
:108A00003BFE3900102210310AA802F035FE290081
:108A1000029A06AB0AA8FFF783FE041E0FD10822B4
:108A200006A908A802F028FE0822311D08A802F0B5
:108A3000A3FD012807D101990398FDF7C9FC28007F
:108A400002F07AFEA3E70124F9E7000070B51C4CA0
:108A500005002368181E10D0002D14D11A78002AA2
:108A60000CD1981C083202F027FE02F045FC0135BB
:108A7000002808D123681D70012070BD0A3318003A
:108A8000082202F019FE2368002BF5D0122002F014
:108A9000D3FC061E0DD0C12321680370457002313E
:108AA0001022023002F008FE23683100587802F0EC
:108AB000ABFB206802F040FE00232360DCE7C046E9
:108AC0009C66FF1FF8B504002020FDF755FB0D4EF6
:108AD000A700BB590500002B0DD000280BD0D8787B
:108AE000FF2809D108492A000C55F35907480333D8
:108AF000611802F0A9FDF8BD290002F025FE00284A
:108B0000F0D1F8E7B866FF1FA066FF1F1D9D00119A
:108B100070B5064D84006359002B05D0D87802F05B
:108B200073FEFF226359DA7070BDC046B866FF1F3E
:108B300070B506008CB00C0015000021302268468C
:108B400002F06AFD31001022684602F095FD1D20FA
:108B500021000322684402F08FFD6846FFF7D8FD2C
:108B60002D21040003222800694402F085FD200025
:108B70000CB070BDF0B50700160097B001931CABA8
:108B80001D7830221EAB00910AA800211C7802F04B
:108B900043FD102239000AA802F06EFD10220021C8
:108BA00002A802F039FD0722310002A802F064FD9C
:108BB000072202AB9818631E9C41019902F05CFDEC
:108BC00002AB9C732B005A1E934102AAD37300215F
:108BD000102206A802F020FD06221D9907A802F027
:108BE0004BFD1A2002ABC01806221F9902F044FD6B
:108BF000102200990EA802F03FFD102202AB0EA930
:108C000008781C78013A6040D2B208700133013113
:108C1000002AF5D10AA8FFF77BFD102212A9040053
:108C20000EA802F049FD102206AB0EA908781D78A7
:108C3000013A6840D2B2087001330131002AF5D1FF
:108C40000AA8FFF765FD044310222098E4B212A998
:108C500002F012FD200017B0F0BD70B50E00140038
:108C60008CB00100102268461D0002F005FD3100A5
:108C7000082204A802F000FD2100082206A802F044
:108C8000FBFC6846FFF744FD04001022280008A9F9
:108C900002F0F2FC20000CB070BDF8B506000D002B
:108CA00000243719AC4200D3F8BD02F0A5FA030A3C
:108CB0003B70631CDBB201379D4203D90234F05490
:108CC000E4B2EEE71C00EDE773B506000C000225E8
:108CD000002819D0002917D0032101A8FFF7DDFFD4
:108CE0006B469A793F231A40013313436A4630009A
:108CF000937101A92200FFF71BFF051E04D1032277
:108D0000E01C01A902F0D8FC280076BD03785807C2
:108D1000DA08C00FD20080009B0710439B0F184356
:108D2000C0B2704707230B40C908C9000B4303704A
:108D30007047000070B50400FFF7EAFE134DA40071
:108D40006359002B21D0186A002801D002F0F4FCEE
:108D50002B59986E002801D002F0EEFC2B59D86EEA
:108D6000002801D002F0E8FC2B59186F002801D030
:108D700002F0E2FC2B59586F002801D002F0DCFC15
:108D8000285902F0D9FC00232B5170BDB866FF1F93
:108D90000E4B8000C35870B50C00002B0FD09D689F
:108DA000002D0CD02B78201D0B706B784B70A97C9C
:108DB000FFF7B8FF2B7E23726B69E36070BD102252
:108DC0000021200002F028FCF8E7C046B866FF1F2B
:108DD000014B18607047C046B466FF1F074A030086
:108DE0008000825810B5002A06D0D088984203D15E
:108DF000012901D1FFF79EFF10BDC046B866FF1FD5
:108E0000F0B5264E95B087000B93BB59050009912C
:108E100012200A92002B31D0D888FFF7A5FB04005E
:108E20001420002C2AD0280010A9FFF7B1FFBB594D
:108E30001E781D6A002E23D00895FDF7EFFA070073
:108E40000020FDF7F1FA0790A379E61D069310AD17
:108E50000CA9089800F0E2FA0EA9280000F0D7FA51
:108E60000B9B0A990493069B09980293079B039610
:108E7000019300970EAB0CAAFFF77CFE15B0F0BD76
:108E8000FDF7CCFA06903000FDF7CEFAE31DA77986
:108E9000079310AB06000893DAE7C046B866FF1FD9
:108EA00030B50C4C85002A59030085B00120002AFA
:108EB0000ED018006946FFF76BFF2B591A78D88837
:108EC000054B002A00D1054B6A46072100F0D9FB6B
:108ED00005B030BDB866FF1F0F9400111D9400113E
:108EE00030B5094C8500295985B0102268462531D6
:108EF00002F0E2FB2A591121044BD0886A4600F0A7
:108F0000C0FB05B030BDC046B866FF1FB994001164
:108F100030B5094C8500295985B010226846353195
:108F200002F0CAFB2A591121044BD0886A4600F08E
:108F3000A8FB05B030BDC046B866FF1FF79400110E
:108F4000F7B54D4F86001020F4590D0002F0A4FA39
:108F5000F3592062186A132200286CD0033A2900C2
:108F60009C6802F0A9FBF3591A780192002A58D1A3
:108F70001E6A227D317B944651400122019F11429D
:108F800001D167461740217D914339432175377BD5
:108F90004F40BC4660460027800701D44F08174069
:108FA000012102208F40227D82433A432275377B84
:108FB0005740BC4660460027400701D497080F4041
:108FC0000420227DBF0082433A432275627D002740
:108FD00094466046727B42400A4201D167460F4088
:108FE0000121627D8A433A436275777B5740BC46D4
:108FF00060460027800701D457080F400220627D99
:109000007F00824317436775767B00227E40760798
:1090100001D4BA080A400426617D9200B1430A4394
:1090200062756A78002A08D06278002A05D0052285
:109030000533DA7700221000FEBD0422297911429F
:1090400005D1A17C114202D10533033AF1E7019A1F
:1090500021782C78002A02D10A002100140018225D
:109060000429E8D8042CE6D805206043034A0533D8
:109070001218525CDDE7C046B866FF1F64BA0011E3
:1090800010B50A001121024B00F0FBFA10BDC046DA
:10909000539500110B0030B587B001AD2B806B46A6
:1090A00004001100981D082202F006FB2A000B2183
:1090B0002000024B00F0E5FA07B030BD7B950011AF
:1090C00010B50A001121024B00F0DBFA10BDC046BA
:1090D000CF95001113B50B0011006A4613706B4653
:1090E00004000622581C02F0E7FA6A460821200014
:1090F000014B00F0C6FA13BDEF95001110B50A0040
:109100001121024B00F0BDFA10BDC0463F96001180
:109110007FB505000B4BAA00D4580800002C0FD0D7
:10912000666F237FE28821780396266F0296E66EAB
:109130000196A46E0094FDF709FC2800FFF7FAFDE4
:109140007FBDC046B866FF1F10B51721FFF7E0FFCF
:1091500010BD000070B50A000D00064B022104008E
:1091600000F08FFA060029782000FFF7D1FF3000C9
:1091700070BDC0461F95001170B586B000236A46C9
:109180001370836804001D78681E0A2859D801A945
:1091900002F06AF9060633373B3F43474B4F530013
:1091A000180000F042F9062312284BD000281BD1EA
:1091B0006088FFF7D9F90823002813D04279002AE4
:1091C00047D1264B1A78072312070BD5244B1A6870
:1091D0000723002A06D01668002E03D0290001AA12
:1091E000B04703006A4613706B461B786088002BFB
:1091F0002AD1FFF767FC06B070BD180000F06CF9CB
:10920000D4E7180000F087F9D0E7180000F093F9D0
:10921000CCE7180000F0ADF9C8E7180000F0C3F97A
:10922000C4E7180000F0F6F9C0E7180000F0F6F9FE
:10923000BCE7180000F013FAB8E7180000F013FAC2
:10924000B4E707236A46137069466088FFF782FF18
:10925000D1E70523012AC5D1024BB8E74565FF1FB9
:10926000B066FF1FB466FF1FF8B52C4F8600F35998
:1092700004000D00002B40D0DA8882423DD15A789C
:10928000062A33D11A78002A2ED0012099681A6A4A
:10929000097D014206D0157B054203D007225A7092
:1092A0000120F8BD0220014204D0157B054201D007
:1092B0000922F4E70420014204D0127B024201D0CB
:1092C0000B22ECE7164B1B68002BE9D05B68002BE8
:1092D000E6D020009847BB5900215B78122BDFD1E4
:1092E0002000FFF715FFDBE70E4BECE7112A04D156
:1092F000002900D032252900F2E7002D08D12000F6
:10930000FFF732F9002803D01023027913430371C9
:1093100021002800FDF798FAC2E7C046B866FF1F93
:10932000B066FF1FB466FF1F70B50E4E8500AB59C7
:109330000400002B13D01B78002B11D10A4B1B68A3
:10934000002B04D05B68002B01D020009847735994
:109350005B78122B03D100212000FFF7D9FE70BDEE
:10936000024BECE7B866FF1FB466FF1FB066FF1F35
:10937000094B8000C3581020002B0CD01A6A002A19
:1093800009D09B68002B06D0127A1B7E101C9A42D3
:1093900000D9181CC0B27047B866FF1F70B5030033
:1093A0000D0014000220002A30D000292ED01370A6
:1093B0000B78081D53704B789370FFF7A7FCE07093
:1093C000012002212B7A23716B7B034063716A7B3E
:1093D0000A401343042263716E7B1640334363716A
:1093E0006E7BF608F600334363712B7B0340A37159
:1093F000287B014000200B43A371297B0A401343C3
:10940000A3712A7BD208D2001343A37170BD10B59B
:109410000A0001000120FFF7C1FF10BD10B50A00CE
:1094200001000220FFF7BAFF10BD70B506000C0066
:109430000220002E30D000292ED07378201D0B7012
:10944000B3784B70F178FFF76DFC01223579257206
:1094500071794B100800134093401040034388106B
:1094600010408000C9080343C9000B436373B179FE
:109470004B100800134093401040034388100240F3
:109480009200C9081343C9000B4321202373FCF742
:1094900073FE854201D2122070BD2220257AFCF78E
:1094A0006BFE8542F7D823781820042BF4D8637814
:1094B000012BF1D80020EFE7030010B502200029AE
:1094C00009D0002B07D00322481C0A7019000D3266
:1094D00002F0F2F8002010BD03000222080010B5CF
:1094E000002B06D0002904D00E32591C02F0E4F8FB
:1094F0000022100010BD030010B50220002909D081
:10950000002B07D00422481C0A7019000C3202F00C
:10951000D3F8002010BD10B5FFF7DEFF10BD03002B
:109520000220002906D0002B04D0052200200A705A
:109530001B784B70704703000220002B08D00029D5
:1095400006D05B7800200B70013B082B00D9183047
:109550007047030010B50220002909D0002B07D066
:109560000622481C0A7019000A3202F0A5F80020F1
:1095700010BD10B5FFF7B0FF10BD02000B000220B8
:1095800010B500290ED0002A0CD0072119701188BF
:1095900059701188090A997011180822D81C02F014
:1095A0008BF8002010BD03000A00022010B5002B2C
:1095B0000CD000290AD0997858780902014311800B
:1095C000901CD91C082202F077F8002010BD03007F
:1095D00010B50220002909D0002B07D00822481C12
:1095E0000A701900921802F067F8002010BD0200FE
:1095F0000B00022010B500290BD0002A09D0092148
:109600001970117818185970511C062202F054F87C
:10961000002010BD10B5FFF75FFF10BD02000B006A
:10962000022010B5002A09D0002907D051781970FE
:1096300011180622581C02F03FF8002010BD03004C
:1096400010B50220002909D0002B07D00A22481C9F
:109650000A701900063202F02FF8002010BD10B574
:10966000FFF73AFF10BD02000B00022010B5002AE0
:1096700006D0002904D018005178FFF753FB0020D2
:1096800010BDF0B585B017001E006A460623050020
:10969000080091819380FEF7C0FC1324011E029004
:1096A0000CD03800B047041E05D1280001A9FEF7F0
:1096B0006FFA041E02D0029802F056F82800FFF755
:1096C00001FA200005B0F0BDF0B504008BB00191A7
:1096D00015000021102202A801F09EFF334EA700C2
:1096E000B85900283CD0C388A34239D10378002B55
:1096F00036D14278062A18D10200010055323531A0
:109700000C3006ABFFF7A9FA002829D12000FFF79B
:109710002FFE020006A902A801F0CEFF200002A938
:1097200001F0AAFD01200BB0F0BD816E002917D019
:109730000B8A112A28D19D420ED101981231093A83
:1097400001F01AFF012807D1BB5920009D6EFFF7D9
:109750000FFE29000200DEE732212000FFF7D8FCCF
:109760002000FEF701FF061E1BD0416A002918D019
:109770000B8AAB4215D108220198123101F0FCFE90
:1097800001280ED1716A0AE09D42E9D108220198B0
:10979000123101F0F1FE0128E2D1BB59996E8A7EA7
:1097A000B9E7200001F058FEBCE7C046B866FF1FCD
:1097B000F0B56B4D87007E5985B0337802900393E6
:1097C000002B00D087E0B368346A019370780628D4
:1097D00017D101221B7D134202D0217B114218D1E7
:1097E0000222134202D0217B114251D104221342A2
:1097F00003D0237B134200D08BE0019B5A7DEB59B1
:1098000091E007380428F8D801F02EFE032E4267B5
:109810008300B36E002B03D11C2001F03DFEB06627
:10982000EB599C6E002C1CD010220021200001F06E
:10983000F3FE0298FFF79CFD01002000FFF72DFAD0
:1098400001F0DAFC2082200008211230FFF725FA0F
:109850000298FFF78DFDA076EB592100D888FFF71D
:109860000FFC0822EB591CE0B36E002B05D01A0048
:10987000198AF0881232FFF70DFC0222019B197D34
:10988000EB5911423DD0207B10423AD0073208E01C
:10989000F488FCF7DBFD01002000FFF711FC0A2231
:1098A000EB595A70029B9C002A595378073B042BB2
:1098B00011D8D088FEF758FE00284ED0C3895A0828
:1098C000D2182849029B0298CB542B5941180433D3
:1098D000254801F0B9FE05B0F0BDFCF79FFD03007F
:1098E0000120834201D100200393EB59DE88FCF76D
:1098F0009BFD039902003000FFF7ECFB019AEB5946
:10990000117D042211420CD0217B114209D00B227F
:10991000C7E7F688FCF73CFD01003000FFF7EEFBDF
:109920006BE7019A527D01210A4204D0607B084214
:1099300001D00C22B5E702210A4204D0607B084224
:1099400001D00E22ADE704210A4204D0627B0A4214
:1099500001D01022A5E71222A3E7FA225200B0E7B5
:10996000B866FF1FBC66FF1F279D001110B5064B90
:109970001A780423100018401A4200D00348FFF759
:1099800027FA002010BDC0464565FF1FE443FF1FB6
:1099900070B50400FFF7D4FA051E43D12000FFF78D
:1099A0007FFA234EA400A0598268937CDB0708D578
:1099B0000321036A1B790B40012B02D1017F0B436A
:1099C0000377431DD97F8B1E022B0DD8022900D0AF
:1099D0000121C088FCF790FF042133591A7F597088
:1099E0000A431A77280070BD01290CD102231022E6
:1099F000437000210C3001F00FFE3059102135303A
:109A0000FFF74BF9EEE70529ECD10223D11843709B
:109A100010220C3001F050FE04233259117F0B4309
:109A20001377EAE708251828DCD1053DDAE7C046B8
:109A3000B866FF1FF0B58BB0059143887E4F9E003E
:109A4000F45915000493002C15D1012902D00020EF
:109A50000BB0F0BD101D57781678FFF757F9EB687B
:109A6000320002932B7A0499019300903B0020006E
:109A7000FCF70CFFEBE7E388049A934201D008203F
:109A8000E6E72378012B00D1D4E0059B581E092876
:109A900000D9CFE001F0E8FC05CE0A29CC506C8556
:109AA0009AB229000498FFF773FFD1E7200029003C
:109AB0001022453001F000FEB9594B78042B02D139
:109AC000013B4B70C3E70B000A00253335320C31E4
:109AD0000498FFF795F90498FFF702FA0522431E50
:109AE0009841BB59C0005A70B2E7200029001022EB
:109AF000553001F0E1FD049B4F4C9D00295904981D
:109B00000A0006AB55320C31FFF77AF929591022B9
:109B1000453106A801F030FD012808D10498FFF76F
:109B2000F7F90590002804D106222B595A700598A0
:109B30008EE708230593FAE763780C2B7AD1E36E5E
:109B4000002B03D11C2001F0A7FCE066BB59D86EA6
:109B500000286FD01022290001F0AEFDBB590498F7
:109B6000DC6EFFF705FC0D22A076BB595A706EE73C
:109B7000E06E00285ED063780D2B5BD12B88082225
:109B80000382A91C123001F097FDBB599A68517DE0
:109B90000222114226D0186A407B104222D00C3299
:109BA000E4E763780E2B45D1236F002B03D11620F9
:109BB00001F072FC2067BB59186F002803D01022F7
:109BC000290001F079FD0F22BB59CFE763780F2BF5
:109BD00030D1206F0622691C103001F06DFDBB5999
:109BE0009A68517D0422114203D0196A497B1142BF
:109BF000D5D100210498FFF78BFA28E7636F002B7B
:109C00000DD0BB59586F0028F3D01022290001F065
:109C100053FD0122BB5952425B6F1A61E9E71420E0
:109C200001F03AFCBB5960675B6F002BE9D126E776
:109C30002978DFE707200BE7B866FF1F10B5064C51
:109C4000207001F0B9FD06212078FDF791FF03484F
:109C5000FEF778FC10BDC046CB66FF1FDD8D0011FE
:109C600000200BB270B50D00834216DA264B18782F
:109C700001F0B2FD041E0DD00378922B0ED0A02B64
:109C800037D0224B1878FF283AD0210001F0BCFAD7
:109C9000002835D180200002684070BD43780E2B2B
:109CA0000BD03E2BEDD18378052B12D0082BE8D1B9
:109CB00081798088FFF7D8FA08E0154B82889A42AC
:109CC000DFD183681878591CFEF7C0FE002817D131
:109CD000D7E7104B1B785B0712D50F4B1B68002B87
:109CE0000ED09B68002B0BD0C289811D80889847BD
:109CF000ECE7FFF741FAA068002801D001F034FD3D
:109D0000200001F019FCC5E7CB66FF1FDD43FF1FF4
:109D1000182000004565FF1FB466FF1F10B50078CE
:109D2000FFF712FA10BD10B50078FFF7FDFA10BD6D
:109D30000C234343084A10B59B185A68002A03D0E5
:109D4000012901D1904710BD9B68002BFBD0002951
:109D5000F9D19847F7E7C046E866FF1F0123834023
:109D6000094A10B5946B1C439463506B984350633D
:109D7000D46B20009843012901D120001843D063FF
:109D8000116B0B43136310BD00800040F0B500243D
:109D90000127154B85B0DA6B144E03921A6C0192B1
:109DA000DA64019BE3403B4217D0039DE5403D4010
:109DB0000295E5B202992800FFF7BAFF316A736A8B
:109DC000002908D03900002B01D0029979402800E1
:109DD000FFF7C4FF01E0002BF9D101340C36172C3A
:109DE000DFD105B0F0BDC04600800040CC66FF1F4B
:109DF000064B01215A68C2400A4204D01B68C34086
:109E00001800084070471B6DF9E7C046008000400D
:109E10000122064B8240002903D0D9680A43DA6048
:109E20007047D9689143D960FAE7C04600380040CE
:109E300030B5032444430F4BE25C1B199C785D78DA
:109E400001232D1B0135AB40013BA340A140DB4367
:109E50000C00122807D808499200521811681940BE
:109E60002143116030BD054A11680B402343136044
:109E7000F8E7C046ABBA001108F0004014F000400B
:109E8000C21F70B5D4B20623092C0BD80125084C8B
:109E90009540002908D00021FFF7CAFF23682B4313
:109EA00023600023180070BD2368AB43F8E7C04669
:109EB00000380040214BF0B51B185B78022B21D1F4
:109EC000032444431E4A1F4EA35C121994780122B6
:109ED00015008540B76B013CE4B23D43A240B56339
:109EE000194C122815D89B0000290CD117495B1872
:109EF00099680A439A600123205C154A83401168DF
:109F00000B431360F0BD11495B1899689143996048
:109F1000F1E70E4B00290DD159690A435A61225CC1
:109F20001328E8D00123203A93400A4908680343E4
:109F30000B60E7E7596991435961F0E7CC66FF1F71
:109F4000ABBA001100800040F0BA001100F00040F0
:109F5000A0F00040A4F00040F8B500241B4E1C4DBA
:109F60001C4B1B5D012B1FD1194A9269E2401A421A
:109F70000BD00122B25693402200143AD2B2022AE8
:109F800009D815494A6913434B61013402360C352F
:109F9000172CE5D1F8BD0022B2560F499200521895
:109FA00091680B439360F0E7022BEED1E7B23800E3
:109FB000FFF71EFF01235840C1B23800FFF77AFFB8
:109FC0003800FFF715FF6877DFE7C0467DBA00115C
:109FD000CC66FF1FCD66FF1F00F000400122023853
:109FE0008240054B002903D059690A435A617047E2
:109FF000596991435961FAE700380040F8B50E00FD
:10A0000001210F008740114A0400D368FD43BB4380
:10A01000D360831E8B4201D8FFF7E0FF00212000B0
:10A02000FFF72EFF0A4A0B4B5168012E05D1394329
:10A030001B1951605E700020F8BD2940516002225A
:10A040001C1962709A6915409D61F4E70038004060
:10A0500000800040CC66FF1F012210B58240074BF4
:10A06000002906D019680A431A600121FFF7C6FFCC
:10A0700010BD196891431960F7E7C04600800040A1
:10A080000C2370B5002543430A4A29009B181D7014
:10A09000094B04001B185D70FFF7B0FF0123A340BC
:10A0A000064928000A681A430A6005490A689A4363
:10A0B0000A6070BDE866FF1FCC66FF1F3480004059
:10A0C0003080004070B504000E00FF2813D0032537
:10A0D0000540FFF7D5FF084AA3089B009B183F22C5
:10A0E000ED00AA40AE401968200091433143196049
:10A0F0000121FFF78DFE70BD18380040F8B50C2423
:10A100004443134B0500E4186368002B03D1A36894
:10A110001220002B1AD0022201270E4B00215B19BE
:10A120005A7028002770FFF769FF63681E1E08D069
:10A13000A3683E00002B04D02800FFF759FE4640DC
:10A14000F6B228003100FFF709FE0020F8BDC04636
:10A15000E866FF1FCC66FF1FF7B5C420FF222B4B1C
:10A1600080001958002491433F3A0A431A50802234
:10A17000274F5202274E1A60274B1D5D002D21D01C
:10A18000A31E012B03D80121E0B2FFF727FF012D09
:10A1900018D11F4B9B69E3402B4213D0E3B2180048
:10A1A0000193FFF725FE01000198FFF755FFE3B289
:10A1B000143B022B1DD801217156184A8D4053695A
:10A1C000AB4353613B7F002B0DD0E5B22800FFF776
:10A1D00095FF2800FFF70CFE7B7F0100834202D031
:10A1E0002800FFF7A5FD01340C370236172CC3D128
:10A1F000F7BD012100237156F3568D40074A9B009D
:10A200009B189A68AA439A60DCE7C04600E100E028
:10A21000CC66FF1F7DBA0011CD66FF1F00F0004025
:10A2200010B501210400FFF7E9FE0123044A0020D4
:10A2300011194B70A34091690B43936110BDC04647
:10A24000CC66FF1F70B50E0015000400FFF718FF65
:10A250000C236343094A20009B189D605E60FFF752
:10A260004DFFF021064B074A8900051E5A5002D0C7
:10A270002000FFF705FF280070BDC046E866FF1FFD
:10A280000000FF1F8D9D001170B5134D07202C7825
:10A29000002C1FD1982221005200280001F064F9FF
:10A2A0000123C420FF222B700C4B80001C635C63D5
:10A2B0000B4B1C605C600B4B195891433F3A0A43AF
:10A2C0001A50802252021A600D20074A074900F0F6
:10A2D000ABFF200070BDC046CC66FF1F0080004071
:10A2E000A0F0004000E100E059A10011599F0011C9
:10A2F000030010B50620072B09D8054A137001F09A
:10A3000073F9D7210020034B034A89005A5010BD2E
:10A310000C44FF1F0000FF1F8D1BFF1F70B51D00A9
:10A3200002240C2910D8094ACA40D2070CD5FBF7E1
:10A330002FFF041E08D1059A04992800FBF744FF5B
:10A34000FCF7B2FDFFF712FB200070BD12100000F9
:10A3500030B50D7802232C009C43184201D02B43CA
:10A360001C0008252300AB43284201D02B002343C7
:10A3700020241D00A543204201D01C4325002A2390
:10A380000D70184204D011781E3B0B43137030BD82
:10A390000028FCD10C2113788B43F7E7F8B51D009A
:10A3A00006AB1B88140007AA0E000B201778002BA1
:10A3B00027D10A78022A49D14A68507811780002D8
:10A3C000244A08438018042840D801F04DF80312AD
:10A3D0001D1B2300F06800F03FFF021CC0B2B84212
:10A3E00000D93A1CD2B22000F1682A8001F064F949
:10A3F00006E00222F3681B882A8023701B0A637020
:10A400000020F8BD0622EEE701232B80F3681B78BD
:10A410002370F5E7F368002B16D008222A801A88EB
:10A4200022701A88120A62705A88A2705A88120A18
:10A43000E2709A8822719A88120A6271DA88A2718F
:10A44000DB881B0AE371DBE72B80D9E701202B8037
:10A45000D7E7C04600D6FFFFF7B516000A781D0003
:10A4600008AB1F880C000123022A18D14A685078D3
:10A47000117800022B4A0843801803280FD800F0F7
:10A48000F3FF02254439E06800F0E6FEC0B207237E
:10A49000B84204D37B190193152B02DD0D2318005C
:10A4A000FEBDE0682A003100C01901F005F96B46D5
:10A4B00000209B88E268D0541B4B1B68834203D06A
:10A4C0001B68834200D098470023E8E70B23002F46
:10A4D000E5D1022DE2D1737832781B021343E26892
:10A4E0001380114B1B68002BEED01B68002BEBD0A8
:10A4F0000120E8E70B23002FD1D1062DCED12A0071
:10A500003100E06801F0D8F8DEE70B23002FC6D158
:10A51000012DC3D132787533012AC0D8E3681A708F
:10A52000D2E7C04600D6FFFFD868FF1F70B50C0009
:10A530001500072837D800F097FF041436361B366D
:10A54000242E182015290BD8184E16220021300071
:10A5500001F062F822002900300001F0ADF800207F
:10A5600070BD18200229FBD11288114B1A80F6E722
:10A5700018200829F4D10A000E48290000F0CCFE6A
:10A58000EDE718200129EBD10B4B10780B49DA6964
:10A59000FFF7DEFEE3E718200129E1D1064B107832
:10A5A0000749DA6BF4E70220DAE7C046C068FF1F0C
:10A5B0008A44FF1F8044FF1F1044FF1F3844FF1FC1
:10A5C0005844FF1F030010B50020DB0704D5072106
:10A5D000024A034800F08CF810BDC04608BB0011C9
:10A5E0001044FF1F054A03001068002803D082882A
:10A5F0009A4201D1806870470068F6E7D06AFF1F71
:10A600000A88030008009A4204D08A8804309A42DB
:10A6100000D0002070470000F8B5F22200230D4F53
:10A620000D4E7968050042433370994200D07B603B
:10A630000A4C0021200000F0EFFF00231A007C608C
:10A64000AB4202D100203370F8BD01332280DBB26F
:10A65000F234F5E7C86BFF1FC66BFF1FD46AFF1FFC
:10A6600073B56B4601900600684615001980FCF72B
:10A670004DFF041E11D1002D0FD07689002E11D070
:10A680000C2000F009FF00280ED0084A046013686F
:10A6900086808560002B02D11060200076BD1A00F4
:10A6A0001B68F7E70224F8E71324F6E7D06AFF1FD8
:10A6B000012100220A4B10B549420A4C19809980A9
:10A6C0009A719A70084B2070012019805A60FFF728
:10A6D000A3FF2078FCF778FF0448FDF733FF10BD97
:10A6E000E068FF1FD06BFF1FC86BFF1F9DA7001105
:10A6F000022310B5002802D0FFF7B2FF03001800B4
:10A7000010BD0000030010B50020DB0704D50421B4
:10A71000024A0348FFF7A4FF10BDC0461CBB00114E
:10A720009044FF1FF0B50E2687B003930CAB1F8833
:10A7300002ABF6180500080031000292FDF768F838
:10A7400004000120002C0FD03088FFF74BFF0300DE
:10A750000E20002B08D05E68002E05D021002800B6
:10A76000039B029A0097B04707B0F0BD0A4B10B5A3
:10A77000984207D10122002352420A808B708A80BE
:10A780008B7110BDFFF73CFF0028FAD001235B421C
:10A79000038000238370F4E7FFFF0000F8B5050095
:10A7A00001290AD1134E00243388F227AB4219D075
:10A7B00028001149FFF7DAFF06E0022904D1013928
:10A7C000FDF73EFF0028EDD0F8BD3B006343726803
:10A7D000D018D35A002B09D03A00002100F01CFFFA
:10A7E0000134E4B2054B1B78A342EED801235B424F
:10A7F0003380DDE7C86BFF1FE068FF1FC66BFF1FDC
:10A8000010B5FFF7FDFE03000020834200D09878CA
:10A8100010BD0000F0B589B01C000EAB80CB0390DA
:10A820001E8810AB1B78049202930B7A0D00DB0696
:10A8300016D42B780593022B24D00498FFF7D2FE70
:10A84000002812D003689C46002B0ED0029B2200E9
:10A85000019329003B00644603980096A04705E059
:10A860000498FFF7BFFE002802D10E2009B0F0BD0A
:10A870008368002BF9D00A22290003989847002802
:10A88000D7D0F3E76B6858781A786B4B0002104307
:10A890009842D2D8043B984210D2684B984242D09A
:10A8A00015D8674BC0180128C7D80B20002EDDD162
:10A8B000EB681A7859683A80200028E0614BC0188C
:10A8C000032800D979E000F0CFFD846A789E5E4BC2
:10A8D0009842B2D10B20002EC8D101233B80EB68F7
:10A8E00031001B7823706889013080B2FCF790FF3B
:10A8F0003A88031E0ED0017802328A183A804289C3
:10A9000062704289120AA27059680278E01C00F055
:10A91000D3FE06E004323A8031000422601C00F0CD
:10A920007BFE0020A2E70B20002E9FD1EB6807A939
:10A930001E8804233B80330A300026706370FCF7C6
:10A9400067FF051E28D004AB9A890E2304A95B1863
:10A950003E49C668FCF7D0FF00280BD12B783C4855
:10A960006A680599FBF786FB002803D1012304AA36
:10A970005B42D3813278022A06D17168201D00F033
:10A980009BFE3B8802333B800E2304AA9B181B8846
:10A99000A3701B0AE370C4E704ABDE81F4E70B206D
:10A9A000002E00D062E7E9680398FFF729FF022331
:10A9B0003B802070000A6070B3E70B20002E00D0AF
:10A9C00054E70222EB681B883A8023701B0A6370ED
:10A9D000A7E7E86800F040FCC2B203000720B242DB
:10A9E00000D243E70DD00299DBB27118994202DB25
:10A9F000921BD3B20293029BE9681A003B8089192B
:10AA00005AE70023F6E70B20002E00D02EE707229E
:10AA1000EB683A801A7822705A7862705A88A2706D
:10AA20005A88120AE2701A792271DA886271DB8818
:10AA30001B0AA37175E7C046042900000228000024
:10AA400000D8FFFFFFD6FFFF03280000FFFF000034
:10AA50004CBA0011F0B58DB06B4600200891202251
:10AA60009B5E83423DDAA64B187800F0B5FE071EC8
:10AA700032D00378B02B2CD10079023816281FD899
:10AA800000F01AFD17001E001E001E0031001E00FF
:10AA900096001E001D011E0052011E0073011E00C3
:10AAA000CD011E0050021E001E001E008E021E0060
:10AAB000E302944B94491B8878880B80FBF71AF8C3
:10AAC0003800FCF79BFF914B1B68002B01D038002E
:10AAD0009847380000F030FD8020089B000243407A
:10AAE00018000DB0F0BDEE220021874800F094FD63
:10AAF0000BAA3B7B7989388900923A000D32FCF72A
:10AB00009FFD0400804B1B78002C3FD146E0804B1A
:10AB1000788805937F4B4100CB5A0BAE073BDBB2E5
:10AB200032880293002301937B4B2100069300930C
:10AB3000059BFFF76FFE744D002810D1069B3A8AE3
:10AB40001B889A420BD138000599123000F014FD91
:10AB5000002804D02B7862899B00EB185A801623BA
:10AB600006A81B18328820007989FCF7C5FE2B78CF
:10AB700004009A00AA1851880029C3D00133DBB21F
:10AB80002B70002807D006A9C98A9180634A1288D1
:10AB90009A42BCD802E0012149429180002B04D0A6
:10ABA00059497888FAF7DAFF8AE73E890A2479E07A
:10ABB00000253E89574B06937B88069A5B009B5A7B
:10ABC000033B9D4202DB002DF0D05BE0162206A87D
:10ABD00012183B7B798900923A0030000D32FCF765
:10ABE0002FFD0590002858D04689017A7888FCF717
:10ABF000F1FC041E44D1464B78880793069B410024
:10AC0000C95A454B0439C9B206AAD28A06930291A1
:10AC1000019400930599079BFFF7FCFD041E2FD1BB
:10AC2000069B39491A88931C002D26D14B807988C0
:10AC3000384B4900CB5A5119033B8B4220DD059B11
:10AC400031485B8941190B71A91C0135C9B2EDB2BC
:10AC5000059145191B0A2B71059B2D4904331818C2
:10AC600000F02AFD2C4B059A1B88D318DDB22C4B23
:10AC70009E4205D00136B6B29CE749889942D6D0AB
:10AC8000002D0CD0204C2800618800F0CDFD2070F4
:10AC900021007888FAF772FF12E7059CF0E7002C94
:10ACA00000D183E77B78142B00D109E716493B7963
:10ACB0004E800B700C717888FAF712FF00E71624AB
:10ACC00006ABE41821003889FCF7A2FD011E00D173
:10ACD000B7E1788822880F4C45002C5B0A4D013C77
:10ACE000E4B2029400240F4B01940095FFF792FD0B
:10ACF000041E00D014E129007888FAF74FFFDFE640
:10AD0000D06BFF1F7C43FF1FE868FF1FDC68FF1F3D
:10AD1000DC69FF1F1865FF1FCC6AFF1F7A43FF1F06
:10AD2000FFFF0000EA68FF1F162406ABE4182100AD
:10AD30003889FCF76DFD011E00D182E178882288F8
:10AD4000AE4C45002C5BAE4D013CE4B202947C89D4
:10AD5000AC4B01940095FFF75DFD041E00D0DFE0D1
:10AD600029007888FAF724FFAAE60025A44B1D8065
:10AD70003B00F6331B78A24A78880792AB4208D989
:10AD80009E4B12880693069943005B5A013B9A42F8
:10AD900003DB0799FAF716FF92E616246B00FB18FF
:10ADA000059306ABE418059B21001889FCF730FDDC
:10ADB000011E03D1059B01241E8973E77888924BFD
:10ADC0002288069C099343001B5B904E013BDBB23B
:10ADD0000293002300960193099BFFF71BFD041EBD
:10ADE00002D0059B1E895DE77B88069A5B009B5A13
:10ADF000079A108832881218934202DC1B1A013B12
:10AE000033807F4C023032880999001900F054FCDD
:10AE10002388328801359B182380EDB2A8E70BAA5E
:10AE20003B7B7989388900923A000D32FCF708FCA7
:10AE300000250590059B002B04D10A24002D00D18C
:10AE40006EE060E0059B7888197AFCF7C3FB01008F
:10AE5000041E63D1694C6C4B788806940993069B59
:10AE60004400E45A694B063CE4B20BAE32880793C7
:10AE70000294019100930599099BFFF7CBFC041EF6
:10AE80004CD1079B5E491B881A1D002D30D14A808A
:10AE9000059B5B4C5A8963191A716B1C9BB2E318B2
:10AEA000120A1A71162306A832881B187989059888
:10AEB000FCF722FDFF21AA1C2E1D03350B00059077
:10AEC00092B2B6B2ADB2002803D006ABDB8AD9B2DB
:10AED0001B0AA218651911712B714C4D301D2A885F
:10AEE0004949201800F0E8FB2B88F618B5B2A1E715
:10AEF0004988914207D17A8806995200525AEB1834
:10AF0000053A9A42C4DC3E4C2800618800F0E4F91E
:10AF1000207021007888FAF75FFED1E5002DF2D18C
:10AF20003E89BFE6162606ABF61831003889FCF7D5
:10AF30006FFC3D000400FA3500282DD0037A9B06F3
:10AF40000CD400227B893989788800923A000C322F
:10AF5000FFF7E8FB041E10D03E8915E03088FFF7AC
:10AF600041FB00281AD08368002B17D02100122241
:10AF700078889847041EE4D0EEE72B78002B02D1A6
:10AF80007888FAF739FE00262B78002B00D097E559
:10AF9000002C00D194E585E60124DDE70E24DBE7F3
:10AFA000162506ABED1829003889FCF731FC041E84
:10AFB00047D0037A9B0611D4154A7B8811889942A1
:10AFC00003D01448814207D11380134BF2261D7819
:10AFD0000023D9B2A94221D30924A1E72888FFF789
:10AFE00001FB00282FD08368002B2CD021001222D7
:10AFF00078889847041EDFD092E7C0461865FF1F87
:10B00000E868FF1FEA68FF1FDC69FF1FCC6AFF1FAB
:10B01000C86BFF1FFFFF0000C66BFF1F31005943C5
:10B02000546801336018615A0029D2D13C000834B9
:10B030002100F22200F040FB21007888FAF7E4FDBD
:10B040003EE501246CE70E246AE71D4B1A887B88D5
:10B050009A4231D07888FAF7E1FD31E5F22305987C
:10B0600051684343CD18C95A00291FD03B7A012BA0
:10B070000BD16C88AB887888AA1D0094FFF752FB2F
:10B08000041E02D000233B722E88F22200212800E9
:10B0900000F0C2FA00232B80059B0133DBB205933D
:10B0A000084B05991B78064A8B42D7D801235B428F
:10B0B0001380002CCED0F5E5002634000596EFE78E
:10B0C000C86BFF1FC66BFF1F70B504000E00150094
:10B0D000FFF796FA031E08D131000548FFF790FAF2
:10B0E00003001120002B02D01C8000209D7070BD39
:10B0F000FFFF0000F8B50B4F06003B780D00140071
:10B10000FF2B0ED00A2000F097F9011E09D0B123C1
:10B110000380002346800371C5800481387800F0E5
:10B1200073F8F8BDD144FF1FF7B50F0008A906005A
:10B13000088809A90B240988002821D10234022B90
:10B140001ED1557813782D021D432B008B4301939C
:10B150007334002B14D1FB68300019000093FFF703
:10B160004FFB019C85420BD02A0030000099FFF76D
:10B17000ABFF041E04D12A0030007989FFF7BAFF23
:10B180002000FEBDF0B50E7885B003900AA80588B2
:10B190000120022E0DD14C682778647824023C43AC
:10B1A000054FBC4205D10398DBB201960095FFF72D
:10B1B000BBFF05B0F0BDC04602290000034B10B52F
:10B1C0001B68002B00D09847FEE7C046D46BFF1FDA
:10B1D00007B501A8FFF7F2FF044A05480021121A3B
:10B1E00000F0C2F9F8F706FBFEE7C046D86BFF1F78
:10B1F000D444FF1F0000000001B40248844601BC93
:10B20000604700BF2951010001B40248844601BCD7
:10B21000604700BF594F010001B40248844601BC99
:10B22000604700BFDD66010001B40248844601BCEE
:10B23000604700BF1531FF1F01B40248844601BCBE
:10B24000604700BF056A000001B40248844601BCA3
:10B25000604700BF8D30FF1F01B40248844601BC27
:10B26000604700BFDD52010001B40248844601BCC2
:10B27000604700BFED4A010001B40248844601BCAA
:10B28000604700BF311B000001B40248844601BC86
:10B29000604700BFCD3BFF1F01B40248844601BC9C
:10B2A000604700BF5D17000001B40248844601BC3E
:10B2B000604700BF156B010001B40248844601BC21
:10B2C000604700BF4D1F000001B40248844601BC26
:10B2D000604700BF090E000001B40248844601BC6B
:10B2E000604700BF090E000001B40248844601BC5B
:10B2F000604700BF5549010001B40248844601BCC3
:10B30000604700BFD91B000001B40248844601BC5D
:10B31000604700BF0124000001B40248844601BC1C
:10B32000604700BF810E000001B40248844601BCA2
:10B33000604700BFB352010001B40248844601BC1B
:10B34000604700BF3939FF1F01B40248844601BC81
:10B35000604700BF8D12000001B40248844601BC62
:10B36000604700BFDD32FF1F01B40248844601BCC4
:10B37000604700BFE117000001B40248844601BCE9
:10B38000604700BF3555000001B40248844601BC47
:10B39000604700BF7530FF1F01B40248844601BCFE
:10B3A000604700BF8552010001B40248844601BCD9
:10B3B000604700BFC521000001B40248844601BCBB
:10B3C000604700BF0139FF1F01B40248844601BC39
:10B3D000604700BF017F000001B40248844601BC01
:10B3E000604700BF9DA9000001B40248844601BC2B
:10B3F000604700BF7536FF1F01B40248844601BC98
:10B40000604700BFB939FF1F01B40248844601BC40
:10B41000604700BF5952010001B40248844601BC94
:10B42000604700BF0D52010001B40248844601BCD0
:10B43000604700BF75A9000001B40248844601BC02
:10B44000604700BF1D4D010001B40248844601BCA5
:10B45000604700BF2124000001B40248844601BCBB
:10B46000604700BF091B000001B40248844601BCCC
:10B47000604700BFE13BFF1F01B40248844601BCA6
:10B48000604700BF5136FF1F01B40248844601BC2B
:10B49000604700BF3119FF1F01B40248844601BC58
:10B4A000604700BF3D4B010001B40248844601BC27
:10B4B000604700BF5522000001B40248844601BC29
:10B4C000604700BFF53BFF1F01B40248844601BC42
:10B4D000604700BF3D18000001B40248844601BC2B
:10B4E000604700BF6571010001B40248844601BC99
:10B4F000604700BF456B010001B40248844601BCAF
:10B50000604700BF4550000001B40248844601BCBA
:10B51000604700BF7939FF1F01B40248844601BC6F
:10B52000604700BF792EFF1F01B40248844601BC6A
:10B53000604700BFE548000001B40248844601BCF2
:10B54000604700BF434D010001B40248844601BC7E
:10B55000604700BFC56D010001B40248844601BCCC
:10B56000604700BF1D4B010001B40248844601BC86
:10B57000604700BFB70E000001B40248844601BC1A
:10B58000604700BFCD4C010001B40248844601BCB5
:10B59000604700BF2D2EFF1F01B40248844601BC46
:10B5A000604700BF0D34FF1F01B40248844601BC50
:10B5B000604700BF8B52010001B40248844601BCC1
:10B5C000604700BF7918000001B40248844601BCFE
:10B5D000604700BF4537FF1F01B40248844601BCE5
:10B5E000604700BF2526000001B40248844601BC24
:10B5F000604700BF8D1BFF1F01B40248844601BC99
:10B60000604700BF6DBC000001B40248844601BC25
:10B61000604700BFF30E000001B40248844601BC3D
:10B62000604700BF154D010001B40248844601BCCB
:10B63000604700BFADAE000001B40248844601BCC3
:10B64000604700BF055E000001B40248844601BCAB
:10B65000604700BFA946010001B40248844601BC0E
:10B66000604700BFC51D000001B40248844601BC0C
:10B67000604700BFF94C010001B40248844601BC98
:10B68000604700BF4551010001B40248844601BC37
:10B69000604700BF691F000001B40248844601BC36
:10B6A000604700BFCD3AFF1F01B40248844601BC89
:10B6B000604700BFB54C010001B40248844601BC9C
:10B6C000604700BFE94C010001B40248844601BC58
:10B6D000604700BFA54F010001B40248844601BC89
:10B6E000604700BFED38FF1F01B40248844601BC2B
:10B6F000604700BF5125000001B40248844601BCE8
:10B70000604700BF4536FF1F01B40248844601BCB4
:10B71000604700BFC9A9000001B40248844601BCCB
:10B72000604700BF851F000001B40248844601BC89
:10B73000604700BF291C000001B40248844601BCD8
:10B74000604700BF014C010001B40248844601BCBF
:10B75000604700BF5147010001B40248844601BC64
:10B76000604700BF2146010001B40248844601BC85
:10B77000604700BFD949010001B40248844601BCBA
:10B78000604700BFE928000001B40248844601BCBC
:10B79000604700BFEDA5000001B40248844601BC2B
:10B7A000604700BFC94A010001B40248844601BC99
:10B7B000604700BFB14E000001B40248844601BC9E
:10B7C000604700BFC926000001B40248844601BC9E
:10B7D000604700BF0519FF1F01B40248844601BC41
:10B7E000604700BFF54E010001B40248844601BC29
:10B7F000604700BF253AFF1F01B40248844601BCE0
:10B80000604700BFA13AFF1F01B40248844601BC53
:10B81000604700BF1147010001B40248844601BCE3
:10B82000604700BFB532FF1F01B40248844601BC27
:10B83000604700BF350E000001B40248844601BCD9
:08B84000604700BFF937FF1F4C
:10B8480000030103020003030402050206020700C5
:10B85800080309030A030B030C000D000E030F0372
:10B86800100311001303140315031603953B00116D
:10B87800C93B001100000000020000008AB8001156
:10B88800192A0F180A000000F1590000FD240000D1
:10B89800414601004D7C0011619C0011B5700011FA
:10B8A800517A00116152001155AA0011BD4E0011C4
:10B8B800A53D0011D53E001100000000161600003D
:10B8C80002000000D4B80011F4FFF3FFD2FC00001E
:10B8D8001540001100000000000000005475796157
:10B8E8000042312E34003030313300676974687596
:10B8F800622E636F6D2F707676780054484232005E
:10B90800020000001CB90011292A282A272A262A01
:10B91800252A242A0A180000E20400007102000007
:10B9280078EC0000744000001027000060F0000070
:10B9380006640000204E0000000000000500000022
:10B948001F501D00023CB400000113001400000049
:10B9580081020000303132333435363738394142CC
:10B96800434445460000000065560011B9560011D1
:10B97800000000000200000088B900116F2A6E2A3A
:10B988001A18000001A00000000000006410B71D94
:10B99800C8206E3BAC30D9269041DC76F4516B6BF5
:10B9A8005861B24D3C7105502083B8ED44930FF0B7
:10B9B800E8A3D6D68CB361CBB0C2649BD4D2D3866D
:10B9C80078E20AA01CF2BDBDFB349B5F80000080BA
:10B9D8000010000000000000B75C00114173001166
:10B9E800DB5C0011497700115F5D00111F770011C2
:10B9F800D55D0011F5760011275E0011BD780011A4
:10BA08008F5E0011BD780011C15E001177780011BA
:10BA1800D55D0011AD7600114D5E0011557800110D
:10BA28000000000000000000335F0011557800118D
:10BA3800955F001159730011052A042A012A002A6A
:10BA48000229032801280028011800180000000016
:10BA58000000000000000000000000870101020152
:10BA680002010102010203030401030101010101B2
:10BA78000303020103000D000E0010001100130063
:10BA88001401070108010A010B011C011D0204022F
:10BA980005020702080219021A021C021D0301030B
:10BAA800020317000201000504000807000B0A0042
:10BAB8001716001D1C010201010504010E0D0111DC
:10BAC80010011413011716011A19020201020B0AB8
:10BAD800020E0D02111002141302171603050403B7
:10BAE8000807030B0A030E0D0001020307090A0BDE
:10BAF8000E0F101112141718191A1B1F20212200DB
:10BB08009DA3001159A400110000000002000000CC
:10BB180052BA00110000000085B1001100000000B9
:08BB28000200000050BA0011F8
:020000041FFFDC
:10000000000000000D3D001190B800118CB80011E7
:100010000462FF1F0000000000000000000000005C
:1000200000000000000000000000000000000000D0
:1000300000000000000000000000000000000000C0
:1000400000000000000000000000000000000000B0
:1000500000000000000000000000000000000000A0
:100060000000000000000000000000000000000090
:100070000000000000000000000000000000000080
:100080000000000000000000000000000000000070
:100090000000000000000000000000000000000060
:1000A0000000000000000000000000000000000050
:1000B0000000000000000000000000000000000040
:1000C0000000000000000000000000000000000030
:1000D0000000000000000000000000000000000020
:1000E0000000000000000000000000000000000010
:1000F0000000000000000000000000000000000000
:1001000000000000000000000000000000000000EF
:1001100000000000000000000000000000000000DF
:1001200000000000000000000000000000000000CF
:1001300000000000000000000000000000000000BF
:1001400000000000000000000000000000000000AF
:10015000000000000000000000000000000000009F
:10016000000000000000000000000000000000008F
:10017000000000000000000000000000000000007F
:10018000000000000000000000000000000000006F
:100190000133FF1F6131FF1FC16601000000000035
:1001A000000000000000000000000000000000004F
:1001B000000000000000000000000000000000003F
:1001C000000000000000000000000000000000002F
:1001D000000000000000000000000000000000001F
:1001E000000000000000000000000000000000000F
:1001F00000000000000000000000000000000000FF
:1002000000000000000000000000000000000000EE
:1002100000000000000000000000000000000000DE
:1002200000000000000000000000000000000000CE
:1002300000000000000000000000000000000000BE
:1002400000000000000000000000000000000000AE
:10025000000000000000000000000000000000009E
:10026000000000000000000000000000000000008E
:10027000000000000000000000000000000000007E
:10028000000000000000000000000000000000006E
:10029000000000000000000000000000000000005E
:1002A000000000000000000000000000000000004E
:1002B000000000000000000000000000000000003E
:1002C000000000000000000000000000000000002E
:1002D000000000000000000000000000000000001E
:1002E000000000000000000000000000000000000E
:1002F00000000000000000000000000000000000FE
:1003000000000000000000000000000000000000ED
:1003100000000000000000000000000000000000DD
:1003200000000000000000000000000000000000CD
:1003300000000000000000000000000000000000BD
:1003400000000000000000000000000000000000AD
:10035000000000000000000000000000000000009D
:10036000000000000000000000000000000000008D
:10037000D1B10011000000000000000000000000EA
:10038000000000000000000000000000000000006D
:10039000000000000000000000000000000000005D
:1003A0000000000000000000000000000D1BFF1F07
:1003B000000000000000000000000000000000003D
:1003C000000000000000000000000000000000002D
:1003D000000000000000000000000000000000001D
:1003E000000000000000000000000000000000000D
:1003F00000000000000000000000000000000000FD
:08183800E06FFF1F4118FF1FC4
:10184000024981F3088802F0BFFB0000E06FFF1F30
:1018500070B500241E491F4A1F484C6308CA1B0567
:101860001B0DE4188242F9D11C4B80228B630021AE
:1018700009201B4B920519621A4B1B4DDA671B4B53
:10188000DA688243DA609A68194802409A60112047
:10189000296002F091F8112002F06EF880226B6C42
:1018A000112093436B64EE23DB006343114A1B0C4E
:1018B00013840122104B9A7201F008FC0F4B1B7825
:1018C000002B04D10E4B1021187802F0F5FA70BDF0
:1018D000000005408805054000060540FF010000A6
:1018E00000F0004004E100E0003800403CF000401F
:1018F000FFDFFFFFD461FF1F8862FF1FB664FF1F79
:10190000B462FF1F10B502F077FA072804D012283E
:1019100008D0022808D010BD044A0420136B0133FC
:101920001363F8E70220F6E71420F4E7C065FF1F11
:10193000F8B507000C0026002500503630785135E8
:10194000002804D10300287058342370F8BD29788A
:10195000CA00481E8141A3183800A25C5B68C9B266
:10196000FFF7D0FF00280DD12B78DA00A218013341
:1019700050602B703378044A013B3370136A013393
:101980001362D8E70123DFE7C065FF1F5C234343F1
:10199000074910B5C9180B0058331B78012B05D126
:1019A000FFF7C6FF034A936A0133936210BDC04636
:1019B000F465FF1FC065FF1F10B502F03DFB064A2E
:1019C0000121130010CB4942D967044B136002F088
:1019D00063F9200010BDC04600E100E010001000D7
:1019E00010B5040002F028FB024B1C6002F054F911
:1019F00010BDC04600E100E0431E5A425341A02200
:101A0000F0B5D2015B421340154D164A40019B18B8
:101A10002A18127E8BB00191002A1BD01A000832BE
:101A2000D46F0022E6B206AFE4B294420EDC28186E
:101A3000C369002B08D0019902AA117106AA049269
:101A400002AA167303A898470BB0F0BD1978B954D1
:101A50000132EAE71A7D1A7806AB01261A70E6E72A
:101A60008068FF1F00400040F0B5254B0400400196
:101A7000C25C85B0002A2BD01A18117E002927D00D
:101A8000917E002924D01179022921D11689D78885
:101A9000D168F51BADB22A1C102D00D9102292B2CC
:101AA000BE4217D11818012303710023C269C380F5
:101AB00003819A4206D068460321037301710293A1
:101AC00001A890470820002C00D0192001F0FEFA50
:101AD00005B0F0BD013C65426C41A0256442ED01BA
:101AE0002C40084D1B186419074D0633013A92B279
:101AF000AA42EDD01888461C1E80085C2070F5E7CD
:101B00008068FF1F00400040FFFF00000F220E4BC7
:101B100010B59868104002380A280BD802F060F817
:101B20000D0A0B0A0A110A0A0A0A060002210020FD
:101B3000FFF762FF10BD0121F9E70020FFF794FFD6
:101B4000F8E7DB6FF6E7C046004000400F220E4B7F
:101B500010B59868104002380A280BD802F040F8F7
:101B60000E0A0B0A0A120A0A0A0A060002210120BA
:101B7000FFF742FF10BD01210800F9E70120FFF740
:101B800073FFF7E7DB6FF5E70090004013B5334CC8
:101B90002378072B3DD8324B1A78324B002A39D1A3
:101BA0008022196852020A431A60252001F0C4FEFF
:101BB00020232D4A11680B43802113606B460422B9
:101BC000C90508680733104228D080210422C905BE
:101BD000C86810422ED080212020C905CA688243DF
:101BE000CA6014221A701A78002A2FD18021C905E0
:101BF000C86820320243CA6014221A701A78002A78
:101C000028D11A4B1A7D22785A601D221A70593237
:101C1000DA6013BD1A6816490A40C5E7086802432E
:101C20000A6014221A701A78002ACED01A78013A63
:101C3000D2B2F7E7C8680243CA6014221A70197852
:101C40004A1ED2B21A700029F9D1C4E71A78013AB3
:101C5000D2B2C7E71A78013AD2B2CEE70C44FF1FDE
:101C6000D444FF1F3CF000400444FF1F002000400C
:101C7000FFFFFEFF564B70B51B68012B03D1554A81
:101C8000936D0133936502F0E7F8534B534A1860A4
:101C9000534B544C1A600123534A1360534A136048
:101CA0002378002B06D006225149524802F024FA2C
:101CB00000232370504A514B10681B78C1B2002B8F
:101CC0000ED14F4CC0B223785BB2002B4FDB237890
:101CD00024785BB264B21B0424021B191B18136026
:101CE0000B1C50294ED95023464A47491078DBB285
:101CF000FF2202284BD10868444C454D267890437A
:101D00002A78964254D9227824782E78023B5D10A6
:101D1000A31B6B435201D31A10335B1118430860A5
:101D200002F07AF9031F012B45D83A4B1B78002BA0
:101D300006D0394B1B78002B02D0002002F024F88B
:101D4000A122364B92009978354B4A431B689B1869
:101D5000832292009B181B78033B012B03D8AF20F2
:101D6000400002F0C1F901222E4BDA8270BD2378C7
:101D700024785BB264B2FF33FF341B0424021B19C6
:101D80000138ABE7CAB2022AAED20223ACE7086838
:101D9000254C264D267890432A78964208D92278F9
:101DA00024782D78023B5B10641B63435201B2E739
:101DB0002378DBB2B2E70228D5D11D4B1B78013B5B
:101DC000022B03D91B4B1B78022BCCD16C20C8E70C
:101DD0009809FF1FFC0FFF1FF864FF1FFF3F000063
:101DE00014100340FC64FF1F0C100340001003405C
:101DF000D50BFF1F7211FF1FB40003408C09FF1F9A
:101E0000680AFF1F490AFF1F94000340460AFF1F8C
:101E1000470AFF1FF908FF1F2209FF1F300DFF1F90
:101E20003409FF1FBC0BFF1F440AFF1F450AFF1F99
:101E30001C09FF1F2309FF1F10B501F03DFF002201
:101E4000014B1A8010BDC046F464FF1F10B502F0AC
:101E50001BF9A121054A89009478054A614312685B
:101E6000044B5218528C1A8010BDC046300DFF1F13
:101E70003409FF1FF464FF1F10B50D4B0D4A99780C
:101E8000A1239B004B431268D218531DD97F0A4BE4
:101E90001B88994209D2441C07D0C82805D0D269B2
:101EA0005B1A5A43054B5343C01802F095F810BD16
:101EB000300DFF1F3409FF1FF464FF1F7102000083
:101EC00070B5244D2B68002B28D002F0F5F82B6854
:101ED000D8402B680400002B27D002F035F82B687F
:101EE000D8401D4B1D4A9978A1239B004B43126893
:101EF000D118D25C91239B00002A20D0CA5801320D
:101F0000CA50174B17491B680868834214D3D23B49
:101F1000181A012A1AD0144B186070BD02F0CCF8C0
:101F2000124B196802F0A0F8D3E702F00DF80F4B3E
:101F3000196802F099F8D4E70D495B18E8E7CA5030
:101F40000C4B1B68DB68E418201AE4E7F530FF301F
:101F5000E1E7C0461C08FF1F300DFF1F3409FF1FBB
:101F60009C09FF1FF864FF1FA009FF1F1808FF1F2F
:101F70002DFF3F000065FF1F70B504000D002829EC
:101F800016D10300A433C2881B889B1A0B4A9BB24C
:101F900093420DD906006A3605223100653001F002
:101FA00013FF002804D13100200001F0F5FF70BDBF
:101FB0002900200001F0B0FEF9E7C046FE7F0000D6
:101FC000F8B50500012001F027FF134CA36AA26AAF
:101FD0009342FBD1114E336001F0A6FF104903007C
:101FE00008601048426894460F4A17680022BC45B2
:101FF00001D24268BA1A0D4802603268AD18A422B4
:10200000E562606A520302436262094A1278002A5A
:1020100001D00F3B0B60F8BD00F00040340AFF1FF9
:10202000E408FF1F28100040180AFF1F1C0AFF1FAA
:102030001C09FF1F70B580241025E405A3682B43FD
:10204000A36002F049F8A368AB43A36070BD000031
:10205000F7B5160080221C001023D205019191686B
:1020600005000B43936000225A4BD7301A6001F0F1
:1020700043FE9D232A002F009B00EB58CA3201210A
:102080000092FC37002B01D00021009A386801F043
:10209000F3FD2900009BCB311A784F4BD3351A60E2
:1020A0004B780A781B0213438A7812041A43CB78C0
:1020B0001B061343494A1BBA13604B790A791B026A
:1020C00013438A7912041A43CB7931001B06134358
:1020D000434A1BBA13606B782A781B021343AA7811
:1020E00012041A43EB781B0613433E4A1BBA1360D3
:1020F000019A330213433C4A13603C4B22001B1BE2
:102100009C4603293DDCB3089A0013005142B21AE1
:10211000032A46D1354AE018511A827840781204D1
:1021200000020243E05C043302430A600022FF2BFA
:102130004BDDF0222E4B12011A600F222D4B1A603C
:102140002D4A1368002BFCD00023224A2749136034
:10215000091B321D0B191B68043A180A23706070A2
:10216000180C1B0EA070E3700434002AF2DC8022ED
:1021700010213B68D20501333B6093688B43936029
:10218000F7BD6346D578981893782D061B042B432A
:10219000157804392B43557804322D022B43036004
:1021A000AFE7022A0AD1114AE05C511AE2185278CC
:1021B000120202430A6004339BB2B7E7012AB5D189
:1021C0000A4A521AE15C1160F5E7084959180A6099
:1021D0000433ACE7000004403C00044038000440F5
:1021E00034000440300004400C000440000104406E
:1021F000040004401000044014000440F7B515002A
:1022000080221C001023D2050091916807000B4327
:1022100093600023654AD730136001F06DFD9D2364
:102220003E009B00F9583B00CA363200FC330029BF
:1022300000D07FE0586801F01FFD390032785C4B18
:10224000CB311A604B780A781B0213438A78AC466C
:1022500012041A43CB78281D1B061343554A1BBA98
:1022600013604B790A791B0213438A7912041A43CB
:10227000CB791B061343504A1BBA13604B7A0A7A78
:102280001B0213438A7A12041A43CB7A21001B06DD
:1022900013434A4A1BBA1360009A2B021343484A5D
:1022A00013602200474B1B1B0093009BCE785B18EA
:1022B00001938B7836061B0433430E78043833437E
:1022C0004E78043136023343019E33600328ECDC40
:1022D0000321A808431C9B002940800003292BD11F
:1022E0003849E5185E18A9786D78E35C09042D0279
:1022F000294319433160030008330021FF2B2DDDF2
:10230000314B324919600F21314B196001232749A4
:102310000B60304B19680029FCD006211B680B406C
:10232000042B20D080220020D20593680A318B43F1
:102330009360FEBD01217DE7022908D121495D1886
:10234000E1184978E35C090219432960D3E70129C0
:10235000D3D11C495918E35C0B60CCE71948181815
:1023600001600433CAE7002310490B606346002B69
:102370000CDC3B00FC335A68102101325A60802289
:10238000D205936801208B439360D2E7009B9B1892
:102390001B68190A13705170190C1B0ED37004239B
:1023A0005B4291709C440432E0E7C0460000044068
:1023B0003C00044038000440340004403000044035
:1023C0000C0004400001044004000440080F000019
:1023D000100004401400044070B5061E19D00222FB
:1023E0005A4B9B799343012B13D1594B1A78FF2AEF
:1023F0000FD15A78FF2A0CD19A78FF2A09D1DA78BE
:10240000FF2A06D11A79FF2A03D15B79FF2B00D16D
:1024100099E0504B0C201A78012A08D000224E4D2A
:102420001A7029780B00093B042B01D8212070BDBC
:102430004B1F012BFAD9454CA37B042B00D982E01A
:10244000A279032A00D97EE09A1ED2B2012A02D8CC
:1024500060881F2877D9002E56D0012E73D1A0880E
:102460000128E3D0002907D1581E032803D801F022
:10247000B7FB121715122E702978481E032811D8A1
:102480000025364B1D602823237501F025FDA84249
:1024900027D0A580CAE702212970EDE70421FBE7D8
:1024A0000321F9E707390129C0D82D490968C96A0C
:1024B0008906BBD52B4908780028B7D1012A01D954
:1024C000002BB3D102230B708021274D26338901C5
:1024D0002878237501F030FC80212878890101F0EB
:1024E000EBFC0123A380214B1B78002B0AD0FA229E
:1024F00080211F4B92001B8809025A431A4B1878FF
:1025000001F042FD002092E701F096FD2B78A680B5
:10251000073B012B03D917482E7001F08DFB114B9F
:10252000114C1A78002A06D08021002220788901D7
:102530001A7001F001FC01F0AFFB80212078090244
:1025400001F0FAFBDEE7122071E7C046A60BFF1F81
:102550006B09FF1F1A09FF1F1C09FF1F4809FF1FF6
:102560000065FF1F2309FF1F1B09FF1F2109FF1F14
:102570002C09FF1F0010004010B5002901D001F008
:102580005BFC10BDF7B5604B01919978A1239B00CE
:102590004B435E4A060014681022E418D6235B0001
:1025A000E0583623FF33E35C00279343222B41D1CD
:1025B000574B0F3A1A600760012501F0DDFB019BC4
:1025C0001880E8235B00E35C002B01D0B34258DDA8
:1025D0000023504FFB70AD33FF33E3581A68002AD5
:1025E00003D09B88DB439B071DD03823FF33E35C7C
:1025F000002B18D09B235B00E35C002B13D1D1335D
:10260000FF33E35CB3420EDAA4235B00E15AE01827
:10261000090A023101F078FB23000122FE33013E5A
:1026200001351A87FA70E8235B00E35C002B2AD09F
:10263000A8B2FEBD03683D00002BBED081880430E7
:10264000090A023101F060FBD6235B00E3581F60EA
:10265000B2E72300B133BA00FF33985801378188BD
:102660000430090A023101F04FFBE8235B00E35C10
:10267000BB42EEDCE822F61AED1800235200A35408
:10268000A6E70027F1E7200001F0EEFB00281FD0AD
:10269000002E1DDD7319882647190193B60020000E
:1026A00001F02AFC5A3080002018406801358188EA
:1026B0000430090A023101F027FB200001F09CFCE4
:1026C000A3590133A351BD4202D0019B9D42E6D1E3
:1026D000114BE35C002BABD095239B00E35C002BFC
:1026E000A6D00E4BE15A0029A2D00D4AA35C994214
:1026F00002D90133A3549BE700231A212000A354DD
:1027000001F022FB94E7C046300DFF1F3409FF1F84
:1027100000140340E010FF1F5A0200007202000084
:102720005E0200000D4970B54A6E0D4CD2038B69F4
:10273000D20BA24206D80B4D0224AA4204D901F0C2
:10274000E3FB70BD02246442E21815007E2425409C
:102750002242F4D0A3432B438B61F0E700F000400A
:102760000A200000FC1C0000F8B51D4B1D4F1A7814
:10277000002A10D1BA7B002A02D101321A7003E07C
:10278000032AFAD0022AF8D001F0A6FB0022012089
:10279000154B1A70F8BD154B154D1C68154B9E78DE
:1027A00001232B702878C0B200F0A2FBBB7B002B6A
:1027B0000BD101F061FCA1239B007343E418832338
:1027C0009B00E41823782B70E4E7032B02D101F07F
:1027D0003BFAF0E70020022BDCD101F03DFCEAE7F8
:1027E0001C09FF1FA60BFF1F2309FF1F3409FF1F32
:1027F000490AFF1F300DFF1FF0B587B00EAD2F78CF
:102800000FAD2D780593AC46634614000E4D0CAA0F
:1028100012782E7803930D9B009201932200059B62
:10282000029701F061FA2E70012C01D0042C08D11E
:10283000802206498B889343054A1278D2011343BC
:102840008B8007B0F0BDC0461C09FF1F6C11FF1F35
:102850007809FF1F0B001B3B70B504003020E02BF4
:102860000DD81300E025493BFF3B9BB2ED00AB4286
:1028700005D8034B200019825A8201F06DFA70BD11
:102880008410FF1F10B501F0E7FA054B00205B68CC
:10289000052B04D9034A5268D20200D4980810BD0F
:1028A00000100040FCE100E070B501F0C5FB0D4BED
:1028B0001B68FC33DC691D6AFFF7E4FF641984427E
:1028C00004D2094B01241B68002B07D004220024EA
:1028D000064B1A70064A93690133936101F0DCF9E3
:1028E000200070BD0065FF1F9809FF1F2309FF1F0F
:1028F000FC0FFF1F70B50C4D2B68FC335C6A01F0B8
:102900009BFBFFF7BFFF2B680025FC339B6AE31896
:10291000834204D2054B1B68AB4200D1051B01F07A
:10292000BBF9280070BDC0460065FF1F9809FF1F56
:10293000D722044B92009B5810B5002B00D098472B
:1029400010BDC0460000FF1F10B501F0D3F8FFF71F
:10295000EFFF2749274BCA6D274C1A4084235B00A1
:102960001343CB65254B1B68186A01F055FA244BBD
:10297000244A1A60244B254A1A60A022244B520094
:102980001A60244B187801F03FFB2000224901F027
:10299000ABFA0023A3600233A360204B20492360DD
:1029A00003232048A36001F09FFA10221E4BFF2052
:1029B0001A60802252031A60802292031A608022D9
:1029C00012041A6001F0E0F9012001F065FAFA2022
:1029D000400001F001FA582001F086FB134801F095
:1029E00073FB012001F0C8FA072001F00DFA10BDB9
:1029F00000F0004000FEFEFF141000400065FF1FC5
:102A0000000003400180063DBC0003403408000084
:102A1000A40003404A0AFF1F71020000C30900001E
:102A2000FFFF3F002810004000E100E0307500008B
:102A3000674E336888331B6883F3088801F004FA13
:102A4000644A6549136800200B401360634B644A75
:102A50001B68934200D1A6E001F056FB0221614AB7
:102A600013688B431360FFF76FFF5F4B5F4C187861
:102A7000C0B201F0F9F80023A3600233A3605C4BFD
:102A80000120236001F0C8F90323A36001F084F959
:102A9000040001F0E1F9050001F07EF9554B1860E2
:102AA00001F0A2F9544B1968621A531EA14200D2D8
:102AB00013008022D203934201D39B029B0A326807
:102AC000D16AC90700D471E04C491C0C09689BB25B
:102AD0004C4359432402090A641803264849FC322E
:102AE00093680A6847489B1A474A0768126847492B
:102AF0009B18474A9A1833409208DB190A60036012
:102B0000042B03D9013233400A6003600E68414947
:102B1000A619300001F0A8FA3F4F3E493B68C318A0
:102B20003B603000019301F0AFF83C4E306808186C
:102B300038493060884205D9019B01333B6001F080
:102B4000A3F8316001F010F9354B1B78002B0DD044
:102B500001F082F9334B621B196812188A4232D293
:102B60004919091B091A304801F0BEF92F4E337A72
:102B7000002B0ED001F070F9621BF168121891421F
:102B800024D94919091B091A294801F0ADF9002374
:102B90003372284B83F3088801F096F8002001F087
:102BA000B3FA01F039F801F0AFFA5CE7DC01990003
:102BB0000234641A5900641A09214B438033CB4014
:102BC000A408E41889E7FA218900CCE71A49DBE771
:102BD0000065FF1F1CF00040FFFFC1FF0C0AFF1F34
:102BE000B641210310000040490AFF1F14100040A5
:102BF000C3090000100AFF1F340AFF1F380AFF1F15
:102C0000200AFF1F280AFF1F1C0AFF1F240AFF1F9C
:102C1000C4090000710200006008FF1F2C0AFF1F9A
:102C20001C09FF1FE408FF1F00100040740BFF1F6A
:102C30003C10004000000020DC050000A022054BF5
:102C400092009B5810B5002B01D0984710BD00F0A2
:102C5000DBFFFBE70000FF1FA122054B92009B5802
:102C600010B5002B01D0984710BD00F0CDFFFBE759
:102C70000000FF1FA222054B92009B5810B5002BAD
:102C800001D0984710BD00F0BFFFFBE70000FF1F19
:102C9000A322054B92009B5810B5002B01D09847FA
:102CA00010BD00F0B1FFFBE70000FF1FA422054BA1
:102CB00092009B5810B5002B01D0984710BD00F032
:102CC000A3FFFBE70000FF1F70B501F0C5F84F4BF5
:102CD000186001F0E1F90400C30702D401F0E4F93F
:102CE00070BD00224A4B1A604A4B187801380428FC
:102CF00029D800F075FF0320181C2400200001F0E3
:102D000053F90128ECD0444C2378042B6ED100F009
:102D10008BFF0028E4D001F0FFF8582001F0E4F91F
:102D200002232370DCE7200000F0BEFFE9E720006B
:102D300001F05AF9E5E7200000F0CEFFE1E72000BE
:102D400001F00AF9DDE701F067F90500012808D173
:102D5000324B1B78053B012B03D82000FFF76EFF99
:102D6000D1E72D4B1B78022B01D0052B20D1022D52
:102D700028D12B4B9B7BAB431CD12000FFF76CFF72
:102D8000264B18780128BED16405BCD424492522DD
:102D90004B7B034205D1233A13405A425341263319
:102DA0001A000B7D9342AED9322001F07DF8AAE7DC
:102DB000022D07D1194B1B78052B11D12000FFF7ED
:102DC00059FFDDE7012D0BD1012B03D12000FFF7C7
:102DD0005FFF98E7062B03D12000FFF767FF92E71C
:102DE000200000F011FF022D8DD1C9E7032B04D183
:102DF0000C4B987C01F0B8F872E7072B00D06FE716
:102E0000094B987B01F010F96AE7C0469C09FF1F47
:102E10009809FF1F9009FF1F2309FF1F1C09FF1FAF
:102E2000A60BFF1FBC0BFF1FD40BFF1FFA210A4B81
:102E30000A4A49001A640A4A5A500A4A04395A503E
:102E4000094A08319A64094A5A50094A5C315A5071
:102E5000084ADA667047C0460000FF1FF927FF1FC7
:102E6000F528FF1FA928FF1FD923FF1F6927FF1F70
:102E7000791EFF1F4D1EFF1F10B500F099FE10BDFB
:102E8000F7B50B0CFF270122009300233C001E0026
:102E90001D009446019089B262469A401000084095
:102EA00018413618B6B2FF2F02D1012E00D19FB2C1
:102EB000009802401A41AD18ADB2FF2C02D1012D8D
:102EC00000D19CB20133102BE6D10320012E07D193
:102ED000012D04D1019B2401E4191C700138FEBDB1
:102EE000102EFCD10238102DF9D00230F7E7000087
:102EF0008023F7B59C46264B264F01932649274A47
:102F0000274D284C284B02281AD1604638600868A3
:102F1000264E3040802636033043086001990978F8
:102F2000002909D11660224A2A60224A2260E02242
:102F300019689143A03A1BE08021C9021160F2E7B1
:102F400066463E600F68194E3E408027FF023E43B2
:102F50000E600199097800290DD1176001280ED162
:102F6000154A2A60154A2260E02219689143C03A46
:102F70000A431A60F7BD802189021160EEE7E02163
:102F80000F4A02432A600F4A22601A688A43F0E718
:102F90004B0AFF1FE0000340D800034090000340AD
:102FA000000003405000034040000340FFFFE3FFE8
:102FB0000280063D804508220180063D8066082289
:102FC0000080069880550822F8B51E4B80261A68A6
:102FD000002014003440324232D11A681A4F324372
:102FE0001A6001223B68063093433B6000F014FFF7
:102FF0000122164D2B681E432E603B680A261343A0
:103000003B608027BF00124B1B683B4211D1013E41
:10301000F6B2FF2E09D17E220E4B1C682B68E40B02
:103020001440934323432B6005E0082000F0F4FE96
:10303000E9E7002EEFD180222B68600893432B60D4
:10304000F8BDC046C4F000405CF0004018F00040FD
:1030500068F0004060F0004010B500F0A5FE0121CE
:103060005820034A00F0F0FFFFF7AEFF10BDC04646
:10307000600AFF1F10B578220021034800F0FCFE13
:1030800000F05AFF002010BD0868FF1F70B5040053
:1030900000F0D2FF00230C200B4A010059438D1889
:1030A000515C00290DD0A14208D1012300246B708E
:1030B00000F03AFE00F0F0FD200070BD01330A2B55
:1030C000EBD11224F6E7C0460868FF1F70B5040074
:1030D00000F0B2FF002319001D000D4A10780028EF
:1030E00006D0A0420CD1557001310C320A29F5D11D
:1030F000002B0AD100F020FF00F0CEFD002070BDB3
:103100005078461EB0411B18EEE700F00DFEF3E7C5
:103110000868FF1FF7B504000C20002384460E4DFD
:10312000019267465F43E85D7E19A04212D00028F5
:103130000BD10A4B9C4662461B7808331370019BE7
:1031400070707C557160B360FEBD01330A2BE8D10D
:103150000320F9E70720F7E70868FF1F0468FF1F4F
:103160008020F8B5484BC0051B68C1248360474BDD
:10317000FF251A68012313434361454BA4001A68D5
:10318000444B40211A60444B1A68444B1A60444B2C
:103190001A59AA431A51C52292009E58AE43314390
:1031A000802699509F583F49F6010F403E439E505C
:1031B0009E5880273602360A3043985080201A598C
:1031C00000020A4002431A5104341A59364E3F0491
:1031D000324080263A431A511A5936061202120A10
:1031E00032431A5108341A5980260A4002431A51B0
:1031F000C32292009F58B446AF4337439F509F5815
:10320000294E0F4007439F509F5837408026360471
:10321000374380269F509F5836063F023F0A374368
:103220009F50C0221F59AF433A431A511A591202F4
:10323000120A1643C6221E5192009C58AC436546A2
:103240002C439C509C5800250C4020439850C7208C
:1032500080001A58154C1140C02212020A431A501D
:10326000134B1B78DB08AB4201DC0020F8BD237850
:10327000002B06D0A368002B00D0984701350C34F2
:10328000EEE71220F2E7C0460844FF1F0444FF1F88
:10329000B0F000400068FF1FB4F00040FC67FF1F63
:1032A00000E100E0FF00FFFFFFFF00FF0868FF1FD5
:1032B0000468FF1F030010B51F2809D8072200204B
:1032C0001340072404490A78A24313430B7010BD2E
:1032D00000230620F5E7C0460468FF1F054B06499A
:1032E0001B780A6805485B0702401B0B134300204C
:1032F0000B6070470468FF1F1CF00040FFFFC1FF18
:1033000070B50C25FFF7EAFF0A4B1C780A4BE4085E
:103310006543ED18002C01D1200070BD2B78002BE7
:1033200006D06B68002B00D09847013C0C3DF1E7BC
:103330001220F2E70468FF1FFC67FF1F1FB5002182
:1033400002220B0001910091052000F035FD0223BF
:103350000B490A681A42FCD120230393039B5A1E8F
:103360000392002BFAD1074A1368002BFCDA0B24D6
:103370006C442000012100F06FFC207804B010BDE7
:1033800090C8004000C8004013B504000A4B0193E8
:10339000019B002B01D1112016BDFFF7CFFF2300A9
:1033A0000340044205D0052000F036FD019B013B9F
:1033B000EDE71800F0E7C046FFFFFF0707B500F094
:1033C0003BFE80220821D205936A0191002B01D196
:1033D0000739916202210C4A11600199481E01903F
:1033E0000029FAD103311160053101910199481E7C
:1033F00001900029FAD11160002B02D18022D20560
:10340000936200F049FC07BD00C00040F0B52D4CB0
:1034100089B02378002B4FD1FEF7CEFA02232A4F32
:1034200003903A681A42FCD120230693069B5A1E49
:103430000692002BFAD1254E3368002BFCDA0120CE
:10344000FFF7A2FF011E02D0112009B0F0BD03005A
:1034500003220190009005AD9F2000F0ADFC0321F8
:10346000280000F0F9FB02233A681A42FCD120231D
:103470000793079B5A1E0792002BFAD13368002B43
:10348000FCDA0120FFF780FF0028DDD10398FEF76A
:10349000A7FAAA786B7811041B020B4329780B4317
:1034A00063601300113B0A49052B07D801239340A1
:1034B000A3600B60012323700020C6E780231B0359
:1034C000F6E7C046F043FF1F90C8004000C8004028
:1034D0009808FF1F1E4B30B55A6818781D4B85B0F1
:1034E000D31859424B4101210093002300F09CFC6A
:1034F000194B1A4A02259A6300221A6510325A653E
:103500008022C4219D65164B1648D202DA678900D5
:103510004258154B80241A4080231B041343435008
:10352000642341200393E40500F006FA402000F0F4
:1035300003FA6562039D6B1E0393002DFAD10323EA
:103540006362FFF73BFFA562FFF760FF05B030BD88
:10355000FC43FF1F95FFFEF700C80040050001FF78
:1035600004E100E000E100E0FFFF00FFF0B585B0FE
:103570000700FEF721FA022305002D4C22681A42AB
:10358000FCD120230093009B5A1E0092002BFAD1FD
:10359000284E3368002BFCDA0120FFF7F5FE0028E7
:1035A00003D01124200005B0F0BD234B236002237B
:1035B00022681A42FCD120230193019B5A1E0192DA
:1035C000002BFAD13368002BFCDA0120FFF7DCFE78
:1035D0000028E6D1194B1F60022322681A42FCD151
:1035E00020230293029B5A1E0292002BFAD13368C9
:1035F000002BFCDA0120FFF7C7FE0028D1D1104BC9
:103600002360022322681A42FCD120230393039BE8
:103610005A1E0392002BFAD13368002BFCDA0120EA
:10362000FFF7B2FE041EBCD12800FEF7D9F9B9E7B6
:1036300090C8004000C8004001000006A8C8004033
:103640000180000110B50020FFF790FF10BD0000C1
:1036500010B5064B18705960FFF73CFF002113208E
:10366000034AFFF757FD002010BDC046FC43FF1F73
:10367000D534FF1FF0B5040085B003920291FEF728
:103680009BF9882263035B0B52051A438023DB05F9
:103690009D6A8023274F0092BA68002601901B0381
:1036A0009A420CD9F82326001B041E401C4206D067
:1036B0008022214B52025E6219680A431A60002D73
:1036C0000BD100F0B9FC02221C4B1A608023DB05F1
:1036D0005A62013A9A6200F0DFFA0023039A934299
:1036E00020D1002D0AD100F0A7FC144B03221D604D
:1036F0008023DB055A629D6200F0CEFA8023BA680F
:103700001B039A4208D9002E06D000220A4B0C490E
:103710005A621A680A401A600198FEF761F900209F
:1037200005B0F0BD009A0299D2181278CA5401333C
:10373000D4E7C046F043FF1F00C8004000C000406F
:10374000FFFFFEFFF0B587B0029103920400FEF781
:1037500033F9019000F070FC802302250122234EF2
:10376000DB0535605D629A6200F096FA204F3B6897
:103770002B42FCD120230493049B5A1E0492002B5D
:10378000FAD11C4D2B68002BFCDA0120FFF7FCFD61
:10379000002802D0112007B0F0BD2000039A029942
:1037A00000F072FB022304003A681A42FCD1202385
:1037B0000593059B5A1E0592002BFAD12B68002B0E
:1037C000FCDA0120FFF7E0FD051EE3D100F034FC38
:1037D00080230322DB0535605A629D6200F05CFAAB
:1037E0000198FEF7FDF8E0B2D5E7C04600C0004002
:1037F00090C8004000C80040F0B5802489B00600A1
:10380000FEF7DAF8E405A36A02250393029000F0BC
:1038100013FC0123304F3D606562A36200F03CFA67
:103820002E4C23682B42FCD120230593059B5A1E66
:103830000592002BFAD12A4D2B68002BFCDA0120CF
:10384000FFF7A2FD002803D01124200009B0F0BD2D
:10385000244B2360022322681A42FCD120230693C2
:10386000069B5A1E0692002BFAD12B68002BFCDA1D
:103870000120FFF789FD021EE6D11B4B03211E60CC
:10388000030001900090202000F096FA02232268A5
:103890001A42FCD120230793079B5A1E0792002B44
:1038A000FAD12B68002BFCDA0320FFF76DFD041E14
:1038B000CAD100F0C1FB80230322DB053C605A62C1
:1038C0009C6200F0E9F9039B002B01D1FFF776FD24
:1038D0000298FEF785F8B8E700C0004090C80040A5
:1038E00000C800400100000694C8004007B500026F
:1038F00001910422000A01A9FFF724FF0EBD000078
:1039000073B5050005240B4AA3005B429B18196898
:103910006B46DE1D3000FFF7B3FA022804D133787E
:103920002B55013CEFD276BD052CFCD00128FAD1F5
:103930000230F8E7140900111F2807D8012380225C
:103940008340D20591680B43936070473F2808D8A5
:103950000123802220388340D20551690B435361F3
:10396000F3E75F28F1D80123802240388340D20555
:10397000116A0B431362E8E71F2807D80122802150
:103980008240C9058B6893438B6070473F2808D8F5
:103990000122802120388240C9054B6993434B6145
:1039A000F3E75F28F1D80122802140388240C90521
:1039B0000B6A93430B62E8E71F2810D880230200AC
:1039C000DB05153A1968012A06D8202291431960AF
:1039D00019680A431A60704701228240F6E73F28BF
:1039E00011D880230200DB05353AD968032A06D8AE
:1039F00010229143D960D9680A43DA60EBE70122CB
:103A000020388240F5E75F28E5D842238022181A43
:103A1000413B8340D205516A99435162516A0B433D
:103A20005362D8E710B50400012813D1A022184929
:103A300092050B685B015B0913430B60154B164A3B
:103A400019681140154A0A431A60402219680A434E
:103A50001A6010BD0028FCD101000A2000F0ACFA69
:103A600021000B2000F0A8FAC0220A4B920019682E
:103A70000A4340211A601A688A431A60B022044936
:103A800012060B685B015B0913430B60E1E7C0465C
:103A900014F000401CF000407F00FEFF80FD01009C
:103AA00072B6074A1368013313600422054B1A608B
:103AB0000023054A13608022D2055360FEE7C0460A
:103AC0007808FF1FC0F00040C4F0004005490B68B3
:103AD000002B05D1044A0A6004490A60044A1360B5
:103AE0007047C046140AFF1F841E0000380AFF1FDB
:103AF000C4F000400023034A1360034A1360034AE2
:103B00001360704754F0004040F1004044F1004021
:103B1000002310B5184C8AB0009301932378012B31
:103B200027D06946012000F0CFF9002817D1009B6B
:103B300012490293019B06AA0393114B02A81B682A
:103B40000493104B1B68059300F0C6FA10220E492F
:103B500006A800F039F9002804D1FF2323700020C3
:103B60000AB010BD0123094A074902A8237000F0DA
:103B7000B3FA0120F4E7C0460465FF1F10290011C5
:103B8000082900110C290011202900110865FF1FC8
:103B900013B501246946012000F096F9034B009407
:103BA0000193FFF7B5FF200016BDC046BB0B000018
:103BB00010B5FFF79FFFFFF7EBFF002802D0024B85
:103BC000984710BDFEE7C046E1A2000002B471466E
:103BD00049084900095649008E4402BC7047C04656
:103BE00002B4714649084900095C49008E4402BC90
:103BF0007047C04603B47146490840004900095A5D
:103C000049008E4403BC704701B40248844601BC9D
:103C1000604700BFE917010001B40248844601BCB7
:103C2000604700BF8552010001B40248844601BCD0
:103C3000604700BF01D7000001B40248844601BCC0
:103C4000604700BFC1A5000001B40248844601BC22
:103C5000604700BF75F8000001B40248844601BC0B
:103C6000604700BF3D71010001B40248844601BCB9
:103C7000604700BF8914010001B40248844601BCBA
:103C8000604700BF2144000001B40248844601BCE3
:103C9000604700BF090E000001B40248844601BC21
:103CA000604700BF9DA9000001B40248844601BCE2
:103CB000604700BF0934010001B40248844601BCDA
:103CC000604700BF8D82000001B40248844601BCF9
:103CD000604700BF7997000001B40248844601BCE8
:103CE000604700BFF535010001B40248844601BCBD
:103CF000604700BF9D6A000001B40248844601BCD1
:103D0000604700BF8944000001B40248844601BCFA
:103D1000604700BFC115010001B40248844601BCE0
:103D2000604700BF51B8000001B40248844601BC9E
:103D3000604700BF21A9000001B40248844601BCCD
:103D4000604700BFB352010001B40248844601BC81
:103D5000604700BF53B9000001B40248844601BC6B
:103D6000604700BF116E000001B40248844601BCE8
:103D7000604700BFD544010001B40248844601BC3D
:103D8000604700BFCD0C010001B40248844601BC6D
:103D9000604700BFED6B010001B40248844601BCDE
:103DA000604700BF156B010001B40248844601BCA6
:103DB000604700BFED68010001B40248844601BCC1
:103DC000604700BF496D010001B40248844601BC50
:103DD000604700BFCD4C010001B40248844601BCDD
:103DE000604700BF8512010001B40248844601BC4F
:103DF000604700BFC166010001B40248844601BCAF
:103E0000604700BFE927000001B40248844601BCB6
:103E1000604700BFF90D010001B40248844601BCAF
:103E2000604700BF0189000001B40248844601BC1C
:103E3000604700BFC56D010001B40248844601BC63
:103E4000604700BFE9D4000001B40248844601BCC9
:103E5000604700BFC9A9000001B40248844601BC04
:103E6000604700BFC95C010001B40248844601BC40
:103E7000604700BF71B0000001B40248844601BC35
:103E8000604700BFB70E000001B40248844601BC81
:103E9000604700BF9573010001B40248844601BC2D
:103EA000604700BF6911010001B40248844601BCAB
:103EB000604700BF6137010001B40248844601BC7D
:103EC000604700BF0D52010001B40248844601BCA6
:103ED000604700BFE1AC000001B40248844601BC69
:103EE000604700BFA9D8000001B40248844601BC65
:103EF000604700BF2D6C010001B40248844601BC3C
:103F0000604700BFD9B0000001B40248844601BC3C
:103F1000604700BFD1AE000001B40248844601BC36
:103F2000604700BF6DF6000001B40248844601BC42
:103F3000604700BFBD5C010001B40248844601BC7B
:103F4000604700BFADAE000001B40248844601BC2A
:103F5000604700BF6D0B010001B40248844601BCFC
:103F6000604700BFF935010001B40248844601BC36
:103F7000604700BF4DF9000001B40248844601BC0F
:103F8000604700BFE512010001B40248844601BC4D
:103F9000604700BF8B52010001B40248844601BC57
:103FA000604700BF85C1000001B40248844601BCDF
:103FB000604700BF0134010001B40248844601BCDF
:103FC000604700BF319E001101B40248844601BC25
:103FD000604700BFD9B1001101B40248844601BC5A
:103FE000604700BF8937010001B40248844601BC24
:103FF000604700BF0534010001B40248844601BC9B
:10400000604700BF5976010001B40248844601BCF4
:10401000604700BFEDA5000001B40248844601BC22
:10402000604700BFDD0C010001B40248844601BCBA
:10403000604700BFC1F7000001B40248844601BCDC
:10404000604700BF75A9000001B40248844601BC66
:10405000604700BF0167010001B40248844601BC0B
:10406000604700BF19FA000001B40248844601BC51
:10407000604700BF090E000001B40248844601BC3D
:10408000604700BFE9F6000001B40248844601BC65
:10409000604700BFF9ED000001B40248844601BC4E
:1040A000604700BFBD0B010001B40248844601BC5B
:1040B000604700BFDD0A010001B40248844601BC2C
:1040C000604700BFE90B010001B40248844601BC0F
:1040D000604700BF8D11010001B40248844601BC55
:1040E000604700BFDD3F000001B40248844601BCC8
:1040F000604700BF7912010001B40248844601BC48
:10410000604700BFE94C010001B40248844601BC8D
:08411000604700BF016C0100D3
:10411800020000004EBA00110100000080B8001132
:10412800020000004ABA0011010000005841FF1FB8
:104138000200000088B80011010000008462FF1F1F
:104148000200000048BA001103000000F861FF1FD8
:1041580012000000020000004EBA00110100000029
:10416800C8B80011020000004ABA0011010000009E
:10417800C5B8001102000000D2B800110300000009
:104188003362FF1F0200000048BA0011030000005C
:104198004862FF1F020000004ABA00110100000037
:1041A800C4B8001102000000D0B8001103000000DC
:1041B8000962FF1F0200000048BA00110300000056
:1041C8002A62FF1F020000004EBA00110100000021
:1041D80008B90011020000004ABA001101000000ED
:1041E800A142FF1F020000001AB9001101000000DF
:1041F80003B90011020000004ABA001101000000D2
:10420800A042FF1F0200000018B9001101000000C1
:104218005062FF1F020000004ABA001101000000AE
:104228009F42FF1F0200000016B9001101000000A4
:10423800F3B80011020000004ABA001101000000A2
:104248009E42FF1F0200000014B900110100000087
:10425800EEB80011020000004ABA00110100000087
:104268009D42FF1F0200000012B90011010000006A
:10427800E9B80011020000004ABA0011010000006C
:104288009C42FF1F0200000010B90011010000004D
:10429800E4B800110202020202020000000000005D
:1042A8000D0C0000E94A0011AD4A00115CB900117B
:1042B80090011D0018001800FFFF07010203040504
:1042C80006020106000000000000000000000000D7
:1042D80000000000000000000000000000000000D6
:1042E80003000000020000004EBA001101000000A7
:1042F8007CB90011020000004ABA00110100000058
:104308005C43FF1F0200000086B900110100000095
:104318007E62FF1F0200000048BA0011030000007F
:10432800E864FF1F020000004ABA00110100000003
:104338005C43FF1F0200000084B900110100000067
:104348008062FF1F0200000048BA0011030000004D
:10435800E064FF1F120000000001000000000111CE
:10436800FFFF000050485936000000000000000020
:104378000B000500F0000000B40000280028002809
:104388003075A000A000A000A00000080008E0010F
:10439800F000100010001000100010001000500075
:1043A8005000500010001000D0070000000000006E
:1043B8000F0001000500307507001000010081FFA3
:1043C80000000000FF00000019700011216E0011AC
:1043D800B16B0011FFFF0100FF000000359A0011CA
:1043E800B1970011C99600110000000000000000FC
:1043F80000000800040000003B0001085902E00129
:1044080088212800FF000000020000004EBA0011B9
:104418000100000014BB0011020000004ABA00119C
:10442800010000008D44FF1F0200000046BA001181
:1044380001000000C068FF1F020000004ABA001116
:10444800010000008C44FF1F0200000044BA001164
:10445800010000008A44FF1F020000004ABA001150
:10446800010000008844FF1F0200000042BA00114A
:10447800010000008044FF1F180018001D00900173
:104488000200000302020000020000004EBA001100
:104498000100000028BB0011020000004ABA001108
:1044A80001000000D044FF1F0200000040BA0011C4
:1044B80000000000000000000200000048BA0011DF
:0A44C80003000000E068FF1F20FF62
:040000051FFF184180
:00000001FF
